:020000040800F2
:10000000A019002045010008111300080311000881
:100010000D130008ED0B0008772200080000000017
:1000200000000000000000000000000003180008AD
:10003000F10B000800000000D91300083519000872
:100040005F0100085F0100085F0100085F01000810
:100050005F0100085F010008F50B0008210C000893
:100060004D0C00085F0100085F0100085F010008F7
:100070005F0100085F0100085F0100085F010008E0
:100080005F0100085F0100085F0100085F010008D0
:100090005F0100085F0100085F010008790C00089B
:1000A0005F010008D91B00085F0100085F0100081C
:1000B0003D1C0008011D00085F0100085F010008E9
:1000C0005F0100085F0100085F0100085F01000890
:1000D0005F010008DD1F00085F01000865200008BF
:1000E0005F0100085F0100085F0100085F01000870
:1000F0005F0100085F0100085F0100085F01000860
:100100005F0100085F0100085F0100085F0100084F
:100110005F0100085F0100085F0100085F0100083F
:100120005F0100085F0100085F0100085F0100082F
:10013000DFF80CD000F010FC0048004791320008B6
:10014000A01900200648804706480047FEE7FEE762
:10015000FEE7FEE7FEE7FEE7FEE7FEE7FEE7FEE777
:10016000391900083101000840EA01039B0703D058
:1001700009E008C9121F08C0042AFAD203E011F8E6
:10018000013B00F8013B521EF9D27047D2B201E0A8
:1001900000F8012B491EFBD270470022F6E710B58C
:1001A00013460A4604461946FFF7F0FF204610BDE5
:1001B000421C10F8011B0029FBD1801A704730B592
:1001C00004460020034600E05B1C934203D2E05C3F
:1001D000CD5C401BF8D030BDF0B480EA0102D40FF2
:1001E0004200B2EB410F02D20246084611464A00D5
:1001F00042D0C30DDDB2C1F3C752AD1A202D35DA9E
:10020000C1F3160141F4000204B15242C5F12006C7
:1002100002FA06F12A411044B3EBD05F23D0C4B1F7
:10022000012DA0EBC35009DCF0BC4FF0004202EA04
:10023000C352DBB200F5000000F02CBA400000F120
:10024000807000EBC350A0F1807040EAD17049008B
:1002500009E0490841EAC071A0EBC35000F5000075
:10026000400800EBC350F0BC00F00BBA6142012221
:1002700002EB4101001BF6E7F0BC704781F0004142
:10028000AAE780F00040A7E780EA010210B502F07B
:100290000043400022D04A001FD0010E01EB126142
:1002A000C0F35600C2F3560240F4000042F40002CC
:1002B000A0FB022000047F39140400D0401C50EA47
:1002C000124001D44000491EC2B20C0604EBD0100B
:1002D000401C4008802A02D003E0002010BD20F01E
:1002E0000100002900DA0020184310BD30B480EA74
:1002F000010202F0004530F0004221F0004013D02E
:1003000090B1C30DD40DC2F31601C0F31600E41A68
:1003100041F4000140F400027D34914201D3641C99
:1003200000E04900002C02DA30BC002070474FF496
:1003300000000023914201D3891A034340084FEA89
:100340004101F7D151B1914202D14FF0004105E096
:1003500002D24FF0010101E06FF0010103EBC45044
:10036000284430BC00F08DB92DE9FE4F81EA03042A
:1003700004F0004421F0004100944FF0000B23F002
:10038000004350EA01045ED052EA03045BD0C3F399
:100390000A54C1F30A552C44A4F2F3340194A0FB8F
:1003A0000254C1F3130141F48011C3F3130343F466
:1003B000801301FB024400FB034E840A970A44EABF
:1003C000815447EA8357A4FB076802958D0A05FB11
:1003D00007854FEA932C04FB0C542705029D4FEA36
:1003E000065847EA1637B5EB08056EEB070C870E83
:1003F000920E47EA811742EA8312A7FB0201B6EB8D
:100400000B0164EB00042B0D43EA0C335E1844EB44
:100410001C50DA465146E7FB0201C5F313044FEACC
:100420000B3343EA14534FEA0432019C43EA0603B8
:10043000A4F10C040294009CCDE900B400F067F92B
:1004400003B0BDE8F08F00200146F9E72DE9F04D3B
:1004500081EA030404F0004B21F0004514464FF0FC
:10046000000A23F0004150EA050220D054EA0102BC
:100470001DD0C5F30A570246C5F31303C1F3130099
:10048000C1F30A5640F4801543F48013A7EB060825
:10049000101BD64608F2FD3873EB050002D308F1B5
:1004A000010801E092185B41B8F1000F03DA002067
:1004B0000146BDE8F08D00204FF4801106468446C9
:1004C0000EE0171B73EB050705D3121B63EB050347
:1004D00006434CEA010C49084FEA300092185B4190
:1004E00050EA0107EDD152EA030012D082EA04007B
:1004F00083EA0501084305D0101BAB4106D2012257
:10050000002306E000224FF0004302E06FF00102FA
:1005100053101AEB06004CEB085110EB0A0041EBAC
:100520000B01BDE8F04D00F0E3B896230022114620
:1005300000F0B0B80EB540F2334102910021CDE990
:1005400000110A460B4600F0E2F803B000BD20F0AF
:100550000040C10DC0F3160040F400007F2901DA0D
:1005600000207047962903DCC1F19601C84070470E
:1005700096398840704700F0004230F000400AD0C1
:10058000C10D01F56071C0F3160042EA0151C208C5
:1005900040071143704700200146704701F00043B7
:1005A00030B421F0004150EA010206D00A0DA2F554
:1005B0006072C1F31301002A02DC30BC00207047D6
:1005C000440F44EAC104C100E01830BC00EBC25043
:1005D00000F057B830B50B46014600202022012418
:1005E00009E021FA02F59D4205D303FA02F5491B01
:1005F00004FA02F52844151EA2F10102F1DC30BD17
:100600002DE9F05F0546002092469B468846064647
:10061000814640241BE0284641464746224600F0DA
:1006200020F853465A46C01A914110D31146184635
:10063000224600F0A3F92D1A67EB01084F46224627
:100640000120002100F09AF917EB00094E41201E0D
:10065000A4F10104DFDC484631462A464346BDE8A2
:10066000F09F202A04DB203A21FA02F00021704793
:1006700021FA02F3D040C2F120029140084319460A
:1006800070470029A8BF7047401C490008BF20F0F0
:100690000100704710B4B0FA80FC00FA0CF050EA88
:1006A000010404BF10BC704749B1CCF1200421FA09
:1006B00004F411FA0CF118BF012121430843A3EB04
:1006C0000C01CB1D4FEA00614FEA102042BF002011
:1006D00010BC704700EBC35010440029A4BF10BCED
:1006E0007047401C490008BF20F0010010BC704753
:1006F00010B5141E73F1000408DA401C41F100012A
:1007000092185B411A4301D120F0010010BD2DE980
:10071000F04D92469B4611B1B1FA81F202E0B0FA77
:1007200080F22032904600F029F904460F4640EA54
:100730000A0041EA0B0153465A46084313D01146BA
:1007400053EA010019D0C8F140025046FFF789FF73
:1007500005460E4650465946424600F00FF90843FA
:1007600005D0012004E020463946BDE8F08D002088
:10077000054346EAE0762C4337430A986305E40ACA
:10078000A0EB08000022FD0A44EA47540A3002D5D3
:1007900000200146E9E7010510196941DDE9084536
:1007A00000196941BDE8F04DA2E72DE9FE4F8046F2
:1007B00081EA0300C00F0C46009021F0004123F0B5
:1007C0000045B8EB0200A94105D2404621469046BB
:1007D0001C460B46024623F00040104347D0270D2D
:1007E000C7F30A00C3F30A510290401A019040284F
:1007F0006BDAC3F3130040F4801B0098924620B1DB
:100800000023D2EB030A63EB0B0B01985946C0F1AE
:100810004002504600F0B2F806460D465046594692
:10082000019A00F0BAF810EB08006141002487EA51
:10083000115284EAE7731A4340D0009A62B3019AD6
:10084000012A4FEA075215DC001B61EB02014FF051
:10085000004202EA0752CDE90042001C41F5801136
:1008600032462B46FFF753FF03B0BDE8F08F4046FA
:100870002146F9E7001B61EB0201001C41F58013E2
:1008800000185B412018A2F5001747EB030140EA6E
:10089000D570B6196D4111E06D084FEA360645EA8C
:1008A000C0754FEA0752001B61EB0201001C41F5C5
:1008B000801149084FEA30000019514132462B4659
:1008C00003B0BDE8F04FFFF713BF009801224000CE
:1008D0000023D0EB020263EBE073009821464FEA5D
:1008E000E074B8EB000061EB0401E9E783F000433A
:1008F0005BE781F0004158E7C1F30A52C1F31301ED
:1009000040F2FF3341F480119A4202DA002001469E
:10091000704740F233439A42A2F2334202DC524221
:10092000FFF79FBE00F02AB830B5041E71F1000435
:1009300004DB4FF00044404264EB0101141E73F1EC
:10094000000405DB1C464FF00043524263EB0403F6
:10095000994208BF904230BD064C074D06E0E06862
:1009600040F0010394E8070098471034AC42F6D3F6
:10097000FFF7E2FB4871000868710008202A04DBD9
:10098000203A00FA02F1002070479140C2F12003A2
:1009900020FA03F3194390407047202A06DBCB1757
:1009A000203A41FA02F043EAE07306E041FA02F32A
:1009B000D040C2F12002914008431946704770B5FB
:1009C0008C1810F8015B15F0070301D110F8013BFA
:1009D0002A1106D110F8012B03E010F8016B01F881
:1009E000016B5B1EF9D12B0705D40023521E0DD4D9
:1009F00001F8013BFAE710F8013BCB1A921C03E027
:100A000013F8015B01F8015B521EF9D5A142D8D35E
:100A1000002070BD21B1826842F00102826003E0D3
:100A2000826822F0010282607047014600208A68D5
:100A300002F004020AB1012000E0002070470146E4
:100A4000C86C80B270470246002013680B400BB19F
:100A5000012000E000207047014600208A6802F073
:100A600008020AB1012000E00020704730B50246BC
:100A70000020002350680F4C20400D790C6844EA98
:100A800005242043506090680B4C2040D1E902546B
:100A90002C434D7944EA450420439060D06A20F409
:100AA00070000C7C641EE4B2234340EA0350D06221
:100AB00030BD0000FFFEF0FFFDF7F1FFF0B504468A
:100AC0000D4600200021092D11DDE068A5F10A0680
:100AD00006EB4607072606FA07F18843A5F10A0642
:100AE00006EB460603FA06F10843E0600CE02069D5
:100AF00005EB4507072606FA07F1884305EB45068F
:100B000003FA06F108432061072A0FDA606B561ECC
:100B100006EB86071F2606FA07F18843561E06EBEA
:100B2000860605FA06F10843606322E00D2A0FDA13
:100B3000206BD61F06EB86071F2606FA07F18843AF
:100B4000D61F06EB860605FA06F10843206310E07F
:100B5000E06AA2F10D0606EB86071F2606FA07F1EA
:100B60008843A2F10D0606EB860605FA06F1084356
:100B7000E062F0BD816841F008018160704721B1F9
:100B8000826842F4A002826003E0826822F4A0023C
:100B900082607047816841F0040181607047000005
:100BA00030B10749096841F40001054A116005E0C8
:100BB0000349096821F40001014A116070470000EF
:100BC0000824014010B501221021024800F094FAD7
:100BD00010BD00000008014010B50022102102489D
:100BE00000F08AFA10BD00000008014000BFFEE7D7
:100BF0007047000010B5012000F072F868B10120C4
:100C000000F068F80548046804E0002108462268FE
:100C100090476468002CF8D100BF10BDA0000020F0
:100C200010B5022000F05CF868B1022000F052F824
:100C30000548046804E0002108462268904764687B
:100C4000002CF8D100BF10BDE000002010B504203A
:100C500000F046F868B1042000F03CF8054804684C
:100C600004E000210846226890476468002CF8D10F
:100C700000BF10BDE800002010B5202000F030F8C3
:100C800068B1202000F026F80548046804E000213F
:100C90000846226890476468002CF8D100BF10BD58
:100CA000F00000200949096829B908490860096865
:100CB000074A116008E005490968814204D00349E8
:100CC000096848600149086070470000DC000020A6
:100CD000E000002001490860704700001404014052
:100CE000014600200022074B1B6803EA0102054B66
:100CF00014331B680B4013B10AB1012000E000203F
:100D00007047000000040140002123498279002A35
:100D10003AD00A46126803689A430B461A600A1DC5
:100D2000126803689A430B1D1A60027911440A681D
:100D300003681A430A60184A0832126803689A4323
:100D4000154B08331A601A1D126803689A43124B38
:100D50000C331A604279102A0ED11A1F12680368E8
:100D60001A430D4B08331A601A1D126803681A43A0
:100D7000094B0C331A600DE00749427911440A68A7
:100D800003681A430A6005E0027911440A6803689F
:100D90009A430A6070470000000401400121034AA1
:100DA000D1700A21B0FBF1F1D16070475C0F0020D7
:100DB0000549897831B90121034A91700A21B0FBB4
:100DC000F1F1D160704700005C0F00200120014963
:100DD000087070475C0F002030B5044604254FF4BE
:100DE000302000F06FF80546042D17D10C4800693B
:100DF00040F002000A49086108464461006940F079
:100E0000400008614FF4302000F05CF805460448CB
:100E1000006941F6FD71084001490861284630BD6E
:100E20000020024004200B49C96801F0010109B10A
:100E300001200EE00749C96801F0040109B1022050
:100E400007E00449C96801F0100109B1032000E07E
:100E500004207047002002400348006940F08000F1
:100E600001490861704700000020024070B5044647
:100E70000D460426F00200F025F80646042E11D196
:100E80000948006940F00100074908612580F00227
:100E900000F018F806460448006941F6FE71084063
:100EA00001490861304670BD0020024002480349F4
:100EB00048600348486070472301674500200240AE
:100EC000AB89EFCD00B502460423FFF7ABFF034625
:100ED00003E0FFF7A7FF0346521E012B01D1002AB2
:100EE000F7D102B90523184600BD000030B5002235
:100EF0008B071C0F0F2303FA04F20B4B8C1053F8D3
:100F000024309343084C8D1044F8253023468C1030
:100F100053F824308C07240F00FA04F42343024CC6
:100F20008D1044F8253030BD080001402DE9F04116
:100F3000024600250026002000230024002791F807
:100F400003C00CF00F0591F803C00CF0100CBCF1BD
:100F5000000F03D091F802C04CEA050591F800C0DB
:100F6000BCF1000F31D0146800202BE04FF0010CD1
:100F70000CFA00F3B1F800C00CEA03069E4220D13F
:100F800083004FF00F0C0CFA03F7BC4305FA03FC87
:100F90004CEA040491F803C0BCF1280F06D14FF0CD
:100FA000010C0CFA00FCC2F814C00AE091F803C06E
:100FB000BCF1480F05D14FF0010C0CFA00FCC2F84F
:100FC00010C0401C0828D1D31460B1F800C0BCF197
:100FD000FF0F34DD546800202EE000F1080C4FF0C4
:100FE000010808FA0CF3B1F800C00CEA03069E42AF
:100FF00021D183004FF00F0C0CFA03F7BC4305FA24
:1010000003FC4CEA040491F803C0BCF1280F05D19D
:1010100000F1080C08FA0CF8C2F8148091F803C02B
:10102000BCF1480F07D100F1080C4FF0010808FA95
:101030000CF8C2F81080401C0828CED35460BDE8DC
:10104000F0810000F0B50A460023002400210025AD
:1010500000F00046B6F1004F02D11D4EF16901E0EB
:101060001B4E7168C0F3034583B200F44016B6F519
:10107000401F08D121F07061154E766826F0706629
:10108000134F7E6012E000F48016B6F5801F06D183
:10109000032606FA05F4A14341F0706106E0460D0F
:1010A000360103FA06F6B14341F0706122B1460DF4
:1010B000360103FA06F6314300F00046B6F1004F60
:1010C00002D1034EF16101E0014E7160F0BD0000FC
:1010D000000001400246002093680B400BB1012044
:1010E00000E00020704702460020D3680B400BB19F
:1010F000012000E0002070470AB1016100E0416179
:10110000704700BFFEE7000001463948417500699D
:1011100028B137480069401E354A106102E00020BE
:10112000334A50703248407D002842D03048C06871
:1011300020B12F48C068401E2D4AD0602C48407D09
:101140002B4A127D90421AD12948807858B12848FC
:10115000C06840B92648807910B90120254A10702E
:101160000120234A90712248C07898B12048C06875
:1011700080B901201F4A10701D4AD0710AE01C4836
:10118000407838B11A48006920B10120194A10701E
:10119000174A50711648007A10B90120154A10708C
:1011A0001348407D124A1075002010710120107202
:1011B00017E00F48007840B10D48007A48B101208F
:1011C0000C4A10700A4A107103E00948407D084A31
:1011D00010750020064AD07090709071D0715071D7
:1011E00010720348007D034A50701046704700009B
:1011F0005C0F00208D01002010B50122082102485B
:10120000FFF77AFF10BD00000008014010B5002272
:1012100008210248FFF770FF10BD000000080140E0
:1012200010B5FFF7F3FF0B48007820F00100401CD9
:10123000084908700121074881811921C1808088EF
:1012400018B90448C08803498880002101480181F9
:10125000418110BD5C01002010B501220821024827
:10126000FFF74AFF10BD00000010014010B500223A
:1012700008210248FFF740FF10BD000000100140A8
:1012800010B5FFF7F3FF0B48007820F00200801C38
:101290000849087001210748018419214183008B06
:1012A00010B90448418B0183002102488183C18326
:1012B00010BD00005C01002008B50820ADF800005A
:1012C00010208DF8030003208DF8020069460D48B8
:1012D000FFF72CFE0820ADF8000010208DF8030069
:1012E00003208DF8020069460748FFF71FFE012220
:1012F00008210448FFF700FF012208210248FFF7F8
:10130000FBFE08BD000801400010014000BFFEE7E1
:101310007047000070B5002100230F22C47804B389
:10132000154C246804F4E064C4F5E064210AC1F1BA
:101330000403CA40447804FA03F18478144021433A
:1013400009010E4C0678A155047804F01F0501240C
:10135000AC4005786D11AD0005F1E025C5F8004100
:1013600009E0047804F01F050124AC40044D067820
:10137000761145F8264070BD0CED00E000E400E079
:1013800080E100E002490143024A11607047000019
:101390000000FA050CED00E010B5FFF713FC002487
:1013A00000E0641C0A2CFCD3FFF716FC002400E0CC
:1013B000641C0A2CFCD3FFF705FC002400E0641C2D
:1013C000C82CFCD3302000F0A5FA002400E0641CF7
:1013D000B4F5FA6FFBD310BD704700000146002042
:1013E000034A506820F440400843506070470000B2
:1013F0000010024029B1064AD2690243044BDA6167
:1014000004E0034AD2698243014BDA61704700006D
:101410000010024029B1064A92690243044B9A61C6
:1014200004E0034A92698243014B9A6170470000CD
:101430000010024030B500210022002400232D4D71
:101440006D6805F00C0121B1042905D0082923D1CC
:1014500005E0294D056022E0274D05601FE0254D80
:101460006D6805F47012234D6D6805F48034022513
:1014700005EB92421CB9214D554305600BE01D4D13
:101480006D6805F400351DB11C4D5543056002E043
:10149000194D5543056002E0174D056000BF00BFC0
:1014A000144D6D6805F0F0010909154D6B5C056878
:1014B000DD4045600F4D6D6805F4E061090A104D8F
:1014C0006B5C4568DD4085600A4D6D6805F46051D0
:1014D000C90A0B4D6B5C4568DD40C560054D6D6804
:1014E00005F44041890B074D6B5CC568B5FBF3F50E
:1014F000056130BD0010024000127A0000093D0075
:1015000048010020580100202DE9F04105460E4613
:101510001746FFF761FB002401E0601CC4B2642C95
:10152000FBDB45F0C005284604F010FA002405E076
:10153000FF2004F00BFA3055601CC4B2BC42F7DB4C
:10154000FFF740FBBDE8F08170B50446FFF744FBB0
:10155000002501E0681CC5B2642DFBDB44F080046B
:10156000204604F0F3F9FF2004F0F0F90646FFF7F7
:1015700029FB304670BD70B50446FFF72DFB0025F2
:1015800001E0681CC5B2642DFBDB44F0C0042046BA
:1015900004F0DCF9FF2004F0D9F90646FFF712FB4E
:1015A000304670BDF8B505460E46362000F0B2F95B
:1015B0003B20FFF7E0FF044604F07F0000B33F202C
:1015C000FFF7C2FF0446B44215DA2C702246691CAC
:1015D0003F20FFF799FF022269463F20FFF794FF63
:1015E0009DF80000094908703A2000F093F99DF831
:1015F0000100C009F8BD3A2000F08CF90020F9E79D
:101600003A2000F087F90020F4E70000E90100200B
:1016100010B5FFF7C1FE01F089FD362000F07AF920
:101620003A2000F077F93B2000F074F9332000F005
:1016300071F9082207493E2000F01FFE064908788C
:10164000FFF782FF04494978884201D000BFFEE7D6
:1016500010BD0000E00100201C71000821B10288CB
:1016600042F04002028004E002884FF6BF731A4045
:10167000028070470246002013890B400BB1012005
:1016800000E00020704701468889704781817047DB
:1016900010B50022028802F441520B884C88234383
:1016A0008C882343CC8823430C8923434C892343D0
:1016B0008C892343CC8923431A430280838B4FF2C6
:1016C000FF74234083830B8A038210BD30B5034629
:1016D0000C461546002207E0184600F008F824F8EA
:1016E00012009B1C501C82B2AA42F5DB30BD0146A1
:1016F000088870472DE9F05F80468A461746B8F1A2
:10170000006F02D33348804501D3BDE8F09FFFF757
:10171000CDFBA8F1006B4FEADB25CBF34909C9F5F6
:101720008064A74200DC3C464DE04FF0006101EBD5
:10173000C5204A142849FFF7C9FF00260BE009EB32
:101740000600254931F810004FF6FF71884200D09D
:1017500003E0701C86B2A642F1DB00BFA6421BDA92
:101760004FF0006101EBC520FFF736FB002608E0D3
:101770003AF8160006EB0901174A22F81100701C0E
:1017800086B2A642F4DB4FF0006101EBC5204A149B
:10179000114900F023F804E022465146404600F08B
:1017A0001DF8A74200D10FE06D1C4FF000090AEBB5
:1017B000440AA044381B87B2B7F5806F02DD4FF4AE
:1017C000806400E03C46B0E700BFFFF745FB00BF88
:1017D0009BE70000000004085C0700202DE9F041B1
:1017E00005460E461746002407E036F81410284632
:1017F000FFF73CFBAD1C601C84B2BC42F5DBBDE8CE
:10180000F081704770B504460D46362000F082F82E
:101810003B2000F07FF82A4621463F2000F02DFDB6
:10182000352000F077F8012070BD10B500F002F807
:1018300010BD00000CB500200190009033480068F6
:1018400040F480303149086000BF3048006800F43F
:10185000003000900198401C0190009818B9019840
:10186000B0F5A06FF1D12948006800F4003010B144
:101870000120009001E0002000900098012843D151
:101880002348006840F010002149086008460068BD
:1018900020F0030008600846006840F0020008607D
:1018A0001A48406819494860084640684860084638
:1018B000406840F4806048600846406820F47C102E
:1018C00048600846406840F4E810486008460068F0
:1018D00040F08070086000BF0C48006800F00070A5
:1018E0000028F9D00948406820F003000749486003
:1018F0000846406840F00200486000BF0348406866
:1019000000F00C000828F9D10CBD000000100240C6
:101910000020024070B50546FFF75EF9002401E0A3
:10192000601CC4B2642CFBDB284604F00FF8FFF700
:1019300049F970BD7047000010B51348006840F0C9
:1019400001001149086008464068104908400E49E6
:101950004860084600680E4908400B490860084680
:10196000006820F4802008600846406820F4FE00EB
:1019700048604FF41F008860FFF757FF4FF000608A
:101980000449086010BD0000001002400000FFF88C
:10199000FFFFF6FE08ED00E0F0B50C46154600220C
:1019A0000021068C4FF6FE773E400684028B018CA8
:1019B0004FF60C7632407E1C06EA03162E43324365
:1019C000104EB0420ED0104EB0420BD0B0F1804F4E
:1019D00008D00E4EB04205D00D4EB04202D00D4E92
:1019E000B04206D14FF6FD76314044F00106314356
:1019F00005E04FF6F576314044F0010631430283AD
:101A00000184F0BD002C014000340140000400407E
:101A100000080040000C0040F0B50C4615460022BE
:101A200000210026078C4FF6EF7C07EA0C0707849D
:101A3000028B018C4FF6FF7707EA041640F6FF474A
:101A40003A404FF6FF7707EA03373A434FF6FF77FE
:101A500007EA05273A43114FB8420ED0104FB8425B
:101A60000BD0B0F1804F08D00E4FB84205D00E4FCA
:101A7000B84202D00D4FB84206D14FF6DF77394059
:101A800046F01007394305E04FF65F77394044F0E0
:101A90001007394302830184F0BD0000002C01408F
:101AA000003401400004004000080040000C0040E9
:101AB000F0B50C461546002200210026078C4FF693
:101AC000FF6C07EA0C070784828B018C4FF6FF77C7
:101AD00007EA04264FF60C773A404FF6FF7707EAFD
:101AE00003172F433A43114FB8420ED0104FB8425C
:101AF0000BD0B0F1804F08D00E4FB84205D00E4F3A
:101B0000B84202D00D4FB84206D14FF6FF573940C8
:101B100046F48077394305E04FF2FF57394044F4EB
:101B20008077394382830184F0BD0000002C01409E
:101B3000003401400004004000080040000C004058
:101B4000F0B50C461546002200210026078C4EF603
:101B5000FF7C07EA0C070784828B018C4FF6FF7726
:101B600007EA043640F6FF473A404FF6FF7707EAA8
:101B700005273A434FF6FF7707EA03373A43114FF9
:101B8000B8420ED0104FB8420BD0B0F1804F08D001
:101B90000E4FB84205D00E4FB84202D00D4FB8429A
:101BA00006D14DF6FF77394046F48057394305E0BA
:101BB00047F6FF57394044F4805739438283018404
:101BC000F0BD0000002C0140003401400004004042
:101BD00000080040000C004010B50121094800F049
:101BE000D4F870B10121074800F0BCF80648046839
:101BF00004E000210846226890476468002CF8D170
:101C000000BF10BD002C0140A80000200949096850
:101C100029B9084908600968074A116008E00549C0
:101C20000968814204D00349096848600149086095
:101C300070470000A4000020A800002010B5082173
:101C4000C80600F0A2F801280ED10821800700F094
:101C500089F81048046804E000210846226890478B
:101C60006468002CF8D100BF0421080700F08DF84B
:101C700001280ED10421800700F074F8064804689A
:101C800004E000210846226890476468002CF8D1DF
:101C900000BF10BDB8000020B0000020094909684D
:101CA00029B9084908600968074A116008E0054930
:101CB0000968814204D00349096848600149086005
:101CC00070470000BC000020C000002010B500F0EC
:101CD000B5FF094801780078401C074A10700529B3
:101CE00009D100201146087004480068401C0349CF
:101CF000086001F06FF910BD94000020280000205A
:101D000010B51021144800F040F801280ED1102120
:101D1000114800F027F81148046804E00021084643
:101D2000226890476468002CF8D100BF01210A485E
:101D300000F02BF870B10121074800F013F80848B3
:101D4000046804E000210846226890476468002C7B
:101D5000F8D100BF10BD000000040040C00000200A
:101D6000C8000020CA430282704721B1028842F0B5
:101D70000102028004E002884FF6FE731A400280DE
:101D800070470146B1F84000704730B50246002068
:101D900000230024158A05EA0103958905EA010458
:101DA00013B10CB1012000E0002030BD70B5054634
:101DB0000C46244885420ED0234885420BD0B5F10D
:101DC000804F08D02148854205D02148854202D065
:101DD0002048854200D100E000BF208850B9238907
:101DE000A28861882846FFF7D7FDE188284600F0E1
:101DF0003CF825E0208804280AD12389A28861883C
:101E00002846FFF709FEE188284600F037F817E07A
:101E1000208808280AD12389A28861882846FFF7EC
:101E200047FEE188284600F036F809E02389A288B9
:101E300061882846FFF784FEE188284600F034F8E0
:101E400070BD0000002C014000340140000400403F
:101E500000080040000C00401AB183890B438381C5
:101E600002E083898B4383817047028B4FF6F373C3
:101E70001A400283028B0A4302837047028B4FF29F
:101E8000FF331A400283028B4FF6FF7303EA0123EC
:101E90001A4302837047828B4FF6F3731A40828392
:101EA000828B0A4382837047828B4FF2FF331A4042
:101EB0008283828B4FF6FF7303EA01231A438283E6
:101EC00070470000002202881D4B98420ED01D4B27
:101ED00098420BD0B0F1804F08D01B4B984205D0F0
:101EE0001A4B984202D01A4B984204D14FF68F7386
:101EF0001A404B881A43174B984207D0164B98420A
:101F000004D04FF6FF431A40CB881A4302808B88D7
:101F100083850B8803850A4B98420BD0094B984266
:101F200008D00E4B984205D00D4B984202D00D4B75
:101F3000984201D10B7A0386012383827047000007
:101F4000002C014000340140000400400008004023
:101F5000000C004000100040001400400040014010
:101F6000004401400048014070B505460C46184841
:101F7000007858BB224629461548401CFEF7F4F865
:101F80001348A0F800410120114908704E1C084672
:101F900090F80011401C00F02FFF98B17078532882
:101FA0000ED100BF0B48006800F4E0600A49084306
:101FB000001D08490860BFF34F8F00BF00BFFEE758
:101FC00000BF00BF032001F071F800BF70BD00002A
:101FD000100200200CED00E00000FA0570B5134877
:101FE000046840F22441124800F081F858B11048CA
:101FF00000F038F9054604E02946002022689047A1
:102000006468002CF8D140F22551094800F06FF8BF
:1020100058B1074800F026F9054604E0294601209A
:10202000226890476468002CF8D170BDD000002071
:10203000003801400949096829B908490860096858
:10204000074A116008E005490968814204D0034944
:10205000096848600149086070470000CC00002012
:10206000D000002070B51348046840F224411248A3
:1020700000F03DF858B1104800F0F4F8054604E0CF
:1020800029460020226890476468002CF8D140F26D
:102090002551094800F02BF858B1074800F0E2F844
:1020A000054604E029460120226890476468002C18
:1020B000F8D170BDD80000200048004021B18289CD
:1020C00042F40052828104E082894DF6FF731A4087
:1020D0008281704702460020B1F5007F00D100BF29
:1020E00013880B400BB1012000E00020704770B551
:1020F0000246002400230025002040F66A16B14263
:1021000000D100BFC1F3421501F01F03012606FAFA
:1021100003F3012D02D19689334006E0022D02D14E
:10212000168A334001E0968A33400C12012606FAE3
:1021300004F41688344013B10CB1012000E00020F3
:1021400070BDF0B50346002400260025002040F6AF
:102150006A17B94200D100BF1846C1F3421401F01A
:102160001F06012707FA06F5012C01D10C3004E007
:10217000022C01D1103000E014301AB107682F434F
:10218000076002E00768AF430760F0BD2DE9F04744
:1021900086B005460E460024A24600BFA146002791
:1021A000B08900B100BF2F462C8A4CF6FF70044066
:1021B000F08804432C82AC894EF6F3100440B088BA
:1021C00031890843718908430443AC81AC8A4FF6D6
:1021D000FF400440B0890443AC8201A8FFF72AF90C
:1021E0001F48874202D1DDF810A001E0DDF80CA005
:1021F000A88900F4004040B10AEBCA0000EB0A10C5
:1022000031684900B0FBF1F807E00AEBCA0000EBC7
:102210000A1031688900B0FBF1F86420B8FBF0F0D7
:1022200004012009642101FB1089A88900F4004001
:1022300040B1322000EBC900B0FBF1F000F0070024
:10224000044308E0322000EB09106421B0FBF1F0F8
:1022500000F00F0004432C8106B0BDE8F0870000B9
:102260000038014001468888C0F308007047C1F378
:1022700008028280704700BFFEE72DE9F041054665
:102280000E461746FEF7A8FC002401E0601CC4B20D
:10229000642CFBDB25F0800545F04005284603F063
:1022A00055FB002404E0305D03F050FB601CC4B219
:1022B000BC42F8DBFEF786FCBDE8F08170B5044651
:1022C0000D46FEF789FC002601E0701CC6B2642EA4
:1022D000FBDB24F08004204603F038FB284603F0A3
:1022E00035FBFEF76FFC70BD7CB5044600201D4633
:1022F000164600290BD0491ECDE90041044B6A4621
:102300002946304600F0DAF8009A002111707CBDB1
:10231000EB2B000802E008C8121F08C1002AFAD1FE
:1023200070477047002001E001C1121F002AFBD155
:10233000704780F3108870472DE9FF5F82B000215D
:10234000DDE90430020DDDF840B0034318D044F657
:102350001050A2F2FF3242431514119801281FD0E9
:10236000A5EB0B00401C5FEA000A4FF000064E4F41
:10237000DFF83891B046504615D5CAF1000413E095
:10238000119801244AA3012801D16FEA0B01029898
:10239000119AC0E90031C0E9024206B0BDE8F09FE1
:1023A000CBF10000DFE704460021404A491842EB28
:1023B0000450CDE9001012E0E00707D032463B465A
:1023C00040464946FDF7D0FF8046894632463B46A7
:1023D00010461946FDF7C8FF06460F466410002C4C
:1023E000EAD1DDE90401DDE90023BAF1000F06DAE4
:1023F000FDF7BAFF42464B46FDF7B6FF05E0FEF794
:1024000025F842464B46FEF721F804460E460022C8
:10241000284BFEF789FA03D84FF0FF30014607E05A
:102420000022254B20463146FEF7BFF9FEF764FA3D
:10243000102409E0002C0ADB0A220023FEF7E0F852
:10244000039B30321A55641E50EA0102F2D1641C1B
:10245000039AC4F111031444119A012A03D00122F2
:1024600008430DD10AE0084304D000204FF0110BBF
:10247000119072E7A3EB0B056D1E0DE05B4504DDCB
:102480004FF0000205F1010504E003DA4FF000020D
:10249000A5F10105002AECD002981199C0E902319A
:1024A000C0E9004579E70000000014400000F03F5B
:1024B000300000000000F0430000E03F2DE9FF4F36
:1024C00095B09B468946064600250FE2252877D120
:1024D00000242746F84A0121059400E0044316F839
:1024E000013F203B01FA03F01042F7D130782A284F
:1024F00011D06FF02F033078A0F13002092A16D8DE
:10250000059A44F0020402EB820203EB42021044FB
:10251000761C0590EFE759F8042B0592002A03DAA0
:10252000504244F40054059044F00204761C307884
:102530002E2816D116F8010F44F004042A280DD0D5
:102540006FF02F023078A0F13003092B09D807EB88
:10255000870302EB4303C718761CF3E759F8047BA3
:10256000761C30786C280FD006DC4C2817D06828F1
:102570000DD06A2814D104E0742810D07A280FD125
:102580000DE044F400140AE044F4801401E044F443
:1025900040147278824202D104F58014761C761CB5
:1025A000307866280BD013DC582877D009DC002857
:1025B00075D04528F6D04628F4D047281AD19DE199
:1025C00018E0632835D0642879D0652812D195E1C8
:1025D000702873D008DC6728F1D069286FD06E2886
:1025E0000DD06F2806D1B5E073282CD0752875D092
:1025F000782874D05A46179990476D1C75E1C4F33A
:102600000250022809D003280DD0D9F80010042860
:102610000DD00D6009F1040967E1D9F80010EA173F
:10262000C1E90052F6E7D9F800100D80F2E70D700D
:10263000F0E719F8041B8DF8001000208DF8010058
:10264000EA46012003E059F804AB4FF0FF30610780
:102650004FF0000102D40DE008F101018846B942B3
:102660000FDA8045F8DB1AF808100029F4D108E0E9
:1026700008F1010188468142FADB1AF808100029A6
:10268000F6D105985B46A0EB080721463846179A15
:1026900000F094FA284400EB080507E04DE029E13A
:1026A0000DE01AF8010B5A4617999047B8F1010846
:1026B000F7D25B4621463846179A13E142E00A22D8
:1026C0000092C4F302524FF0000A022A08D059F8CF
:1026D00004CB032A4FEAEC710AD00DE029E02AE08E
:1026E00009F1070121F00702F2E802C1914609E071
:1026F0000FFA8CFC4FEAEC71042A03D14FFA8CFCE0
:102700004FEAEC71002907DA0A460021DCF1000CDF
:1027100061EB02012D2202E0220504D52B228DF867
:102720000420012203E0E20701D02022F7E79046CF
:1027300059E00A2102E010220DE010214FF0000ABA
:1027400000910BE010224FF0000A44F00404082727
:10275000009203E008224FF0000A0092C4F30252F4
:10276000022A05D059F804CB0021032A08D009E039
:1027700009F1070121F00702F2E802C1914605E0E4
:102780001FFA8CFC042A01D10CF0FF0C4FF000085A
:10279000220728D5702806D0009B83F0100353EA47
:1027A0000A0305D00EE040228DF80420012208E043
:1027B0005CEA010206D030228DF804208DF8050075
:1027C00002229046009B83F0080353EA0A030AD1D1
:1027D0005CEA010201D1620705D530228DF80420A0
:1027E0004FF001087F1E582804D034A003900EA893
:1027F00002900DE036A0F9E753466046009AFDF7D7
:10280000FFFE84460398825C0298401E029002708C
:102810005CEA0100F0D1029806A9081A00F1200A2A
:10282000600702D524F4803400E00127574502DD1B
:10283000A7EB0A0000E0002000EB0A0100900598D9
:102840004144401A0590E00306D45B462146179A9E
:10285000059800F0B3F90544002706E001A85A46A0
:10286000C05D179990476D1C7F1C4745F6DBE00360
:102870000CD55B462146179A059800F09FF9054450
:1028800004E030205A46179990476D1C0099481E65
:1028900000900029F5DC08E0029802995A46007879
:1028A000491C0291179990476D1CBAF10001AAF1D9
:1028B000010AF1DC65E10000092801003031323302
:1028C000343536373839616263646566000000006C
:1028D0003031323334353637383941424344454656
:1028E0000000000000F058F90544761C30780028FC
:1028F0007FF4ECAD19B02846BDE8F08F620700D434
:10290000062709F1070222F0070CFCE80223E14642
:1029100003F000485FEA080C02D00FF2702C0DE0C3
:102920005FEA045C02D50FF2682C07E05FEAC47C22
:1029300002D00FF2602C01E0AFF2700C4FF0FF38C4
:1029400023F00043CDF850C065280CD006DC4528A4
:1029500009D046281DD047283DD13DE0662818D033
:1029600067287ED138E00021112F01DB112000E023
:10297000781CCDE9000106A90EA8FFF7DDFCDDE912
:102980000F010E9A03910021009207F1010A0491B0
:102990004DE04FF000400097CDE9011006A90EA8C8
:1029A000FFF7CAFCDDE90F0203920E9B119900228A
:1029B000DDF80CA00093049211B9791C00EB010A18
:1029C000B7EB0A0004D4C0F1FF3007F1010A04900C
:1029D000AAEB0700019044E0012F00DA0127002153
:1029E000112F01DD112000E03846CDE9000106A9D4
:1029F0000EA8FFF7A1FCDDE90F010E9A039100215B
:102A000004910092BA4621070CD40399514500DA8B
:102A10008A46BAF1010F05DD009AAAF10101515C65
:102A2000302908D0B84202DA10F1040F06DA012189
:102A3000CDE9011015E0AAF10101E9E7002805DC64
:102A4000049901440491AAEB000102E0411C5145A4
:102A500000DD8A460499401A401C01904FF0004066
:102A60000290200704D40198504501DBCDF8048082
:102A700000208DF84F0002980DF14F07B0F1004F84
:102A800025D02B200E9002984FF0020800280CDA77
:102A9000404202902D200E9007E00A210298FDF797
:102AA00099FD3031029007F8011DB8F10001A8F13D
:102AB0000108F2DC02980028EFD1791E0E98087008
:102AC000307800F0200040F0450007F8020D12A811
:102AD000C01B00F107081498007800B1012000EB3A
:102AE0000A01019801EBE07105984144401A401E2B
:102AF0000590E00306D45B462146179A059800F03E
:102B00005DF805441498007818B15A461799904713
:102B10006D1CE00324D55B462146179A059800F00A
:102B20004DF805441CE00498002807DBDDE90301AB
:102B3000884203DD0098405C179901E01799302026
:102B40005A469047049805F10105401C04900198ED
:102B5000401E019004D12E205A46179990476D1CB3
:102B6000BAF10001AAF1010ADDDC05E017F8010B5A
:102B70005A46179990476D1CB8F10001A8F1010859
:102B8000F4DC5B462146179A0598ABE62D00000061
:102B90002B000000200000002DE9F0410446002534
:102BA0001E461746880404D405E039462020B04765
:102BB0006D1C641EF9D52846BDE8F0812DE9F04171
:102BC000044600251E469046C80301D5302700E084
:102BD0002027880404D505E041463846B0476D1CDF
:102BE000641EF9D52846BDE8F0814A68002A06D05F
:102BF0000A68531C0B6010704868401E486070479C
:102C000008B54FF48050ADF8000010208DF8030097
:102C100003208DF8020069460448FEF787F9002278
:102C20004FF480510148FEF767FA08BD00080140E3
:102C3000C8200149088070478801002010B563480A
:102C40000078401C6149087008460078604909789E
:102C5000884215DB00205D4908705E48008878B125
:102C60004FF480515C48FEF73EFA08B9012000E0BD
:102C70000020044622464FF480515748FEF73CFAA4
:102C80005448008868B153480088401E5149088064
:102C90000846008828B900224FF480514E48FEF7BC
:102CA0002BFA00248EE004EB84014C4830F821001C
:102CB000002858D004EB8401484830F82100401E19
:102CC00081B204EB8402454820F8221004EB840111
:102CD00030F82100002874D104EB84013F4800EB58
:102CE0008100008900286CD004EB84023B4901EB91
:102CF00082010869804704EB8401384800EB8100B9
:102D00000089401E81B204EB8402344800EB82004B
:102D1000018104EB8401314800EB81000089A8B9EE
:102D20002E48001F00780121A14088432B49091F2C
:102D3000097860F300012948001F0170002104EBAD
:102D40008402001D00EB820081803AE004EB8401E4
:102D5000224800EB8100C18804EB84021F4800EB8D
:102D6000820081802DE004EB84011C4800EB81008F
:102D7000808830B304EB8401184800EB8100808820
:102D8000401E81B204EB8402144800EB8200818073
:102D900004EB8401114800EB8100808888B904EBC2
:102DA00084010E4800EB8100418804EB84020B484B
:102DB00020F8221004EB8402014601EB820108692D
:102DC0008047641C022CFFF66EAF10BD8B01002003
:102DD0008A010020880100200008014060010020D5
:102DE00001490870704700008A0100203C20014919
:102DF00008807047880100202DE9F04304460D4605
:102E00000027267894F8018014F80690681EB042D6
:102E10000CD108F0800040B9681E81B24A462046B5
:102E200000F00EF810B1012700E001273846BDE898
:102E3000F083000000200149887070475C0F00207B
:102E400070B505460E4614460723552231462846DE
:102E500000F006F8A04201D1012070BD0020FCE77F
:102E6000F0B50446104611E014F8016B70400025DF
:102E70000AE000F080061EB14606300E584001E020
:102E80004606300E6E1CF5B2082DF2DB0E1EA1F1C7
:102E90000101E9D1F0BD30B504460D463123FF22D2
:102EA00029462046FFF7DCFF30BD70B505460E46CB
:102EB00014463123FF2231462846FFF7D1FFA042B6
:102EC00001D1012070BD0020FCE7000010B5404892
:102ED0000068007800B910BD00203D4909680870FD
:102EE0003B480068407806286DD2DFE800F06C248B
:102EF000033E155800F00EF938B1FFF79BFFFDF7C0
:102F000065FF012001F06CF805E000F009F910B947
:102F10000520FDF74DFF57E000F0FCF820B1FFF76A
:102F200089FFFDF753FF05E000F0FAF810B905201E
:102F3000FDF73EFF48E000F0DDF830B11E20FDF760
:102F40002DFF012000F0DEFD0EE000F0E9F828B1D1
:102F5000FFF74CFF012000F0D5FD05E0FDF736FF3F
:102F60004FF49670FDF71AFF2EE000F0C3F830B171
:102F70001E20FDF713FF002000F0C4FD0EE000F05E
:102F8000CFF828B1FFF732FF002000F0BBFD05E0CD
:102F9000FDF71CFF4FF49670FDF700FF14E000F002
:102FA000B9F848B1FFF746FFFDF710FFFFF71EFF26
:102FB000002001F015F805E000F0B2F810B9052086
:102FC000FDF7F6FE00E000BF00BF00BF83E7000092
:102FD00000000020002034E000EB40011A4A02EB20
:102FE0008101896861B300EB400102EB810149680E
:102FF000491C00EB4002144B03EB8202516000EBD2
:10300000400203EB82029268521E914218D30021C3
:1030100000EB400203EB8202516000EB40011A46D4
:1030200012F8211029B9002100EB400203EB8202C3
:10303000916001218140054A12681143034A1160E1
:10304000401C2028C8DB70479C0F0020A8010020EE
:1030500010B504460120FFF76CF9002004EB440191
:10306000074A02EB8101886004EB440102EB810115
:10307000486004EB440102F82100FFF75AF910BD43
:103080009C0F002010B500240120FFF752F90548DD
:10309000046805480460002002490860FFF749F908
:1030A000204610BDA8010020AC01002010B5044648
:1030B0000120FFF73EF9002004EB44010B4A02EB2C
:1030C0008101886004EB440102EB8101486004EB5C
:1030D000440102F821000120A04005490968084385
:1030E000034908600020FFF724F910BD9C0F002061
:1030F000A80100200148C079704700005C0F002043
:10310000014601208840024A1268104070470000C2
:10311000AC01002001488079704700005C0F00205E
:1031200001480079704700005C0F002010B50024B2
:103130000AE0074A02EB44025178054A12F81400EB
:10314000FFF7BCF8601C84B2162CF2D310BD00004F
:103150001C71000810B5002401211248FDF7BAFFC8
:1031600008B901241CE04FF480410F48FDF7B2FF7D
:1031700008B9022414E04FF400410B48FDF7AAFF00
:1031800008B903240CE040210848FDF7A3FF08B963
:10319000042405E080210548FDF79CFF00B90524C3
:1031A000204610BD00080140000C01400010014005
:1031B00008B50120ADF8000048208DF803006946ED
:1031C0001648FDF7B3FE4FF48040ADF800004820EC
:1031D0008DF8030069461248FDF7A8FE4FF4004041
:1031E000ADF8000048208DF8030069460C48FDF753
:1031F0009DFE4020ADF8000048208DF80300694690
:103200000848FDF793FE8020ADF8000048208DF8B7
:10321000030069460348FDF789FE08BD0008014028
:10322000000C01400010014070B504460D46142208
:103230000B49A1F11400FCF797FF1422084914313F
:103240000748FCF791FF142105481430FCF7A5FF4F
:103250001422214602481430FCF786FF70BD00009E
:103260007415002070B504460D4614220749A1F1DB
:103270001400FCF779FF14210448FCF78EFF142298
:1032800021460248FCF770FF70BD00007415002055
:103290004FF4A060FEF776F802F0FCFD0121FE4835
:1032A000FDF7D0FE0B21FD4801F052FFFB48827A6A
:1032B0000A21FFF7FAFD48B9F848F9490A6802609F
:1032C0004A6842600A890281897A8172FFF770FF39
:1032D000FDF7F2FFF3494FF4E13002F059FDF249F6
:1032E000C82002F017FD00F0BFFBFFF789FCEB4997
:1032F000487AFFF775FDE949087A02F093FCEB493B
:10330000002002F005FCE549087902F0D1FCE34910
:1033100091F90610E64A505602F0DCFCDF49C87904
:1033200002F074FCE34801F03BF8DC49097A01EB58
:103330008101E14A02EB810001F0FCF9D7490979EA
:10334000D64A527911FB02F101EB8101490001EBF0
:103350004102C2EBC111D14A127AD84B53F8222054
:1033600002EBC10001F0F0F9CC4991F90610D04A06
:10337000505601F02BFAC949C979D14A52F82100B7
:1033800001F004FAC548017A04230022104601F036
:103390000DF9C24801791F230022012001F006F92E
:1033A000BE48417915231422022001F0FFF8BB48E2
:1033B00090F9061009230022032001F0F7F8B7481E
:1033C000C17907230222042001F0F0F8B3490979FA
:1033D000B24A527911FB02F101EB8101490001EB84
:1033E0004102C2EBC111AD4A127AB44B53F822200C
:1033F00002EBC10001F058FDA849497901EB8101B8
:1034000049004FF47A7211FB02F001F047FDA34925
:10341000097A01EB8101A84A02EB810001F056FD17
:103420009E49C979A64A52F8210001F043FD9B4903
:1034300091F906109E4A505601F042FD012001F01C
:10344000C9F8A0A001F0C0F8FFF7F2FB0A220121A1
:10345000002002F08FFD4FF4FA720121084602F0BD
:1034600089FD02F0BBFB95E2FFF70CFE9A4908804C
:103470000020FFF745FE38B198480078FDF744FE7C
:1034800097490860FFF722FD0120FFF739FE60B37E
:1034900000F0C0FA83469349FCF728FF8246FDF707
:1034A0006AF806460022904BFCF7D0FF0446002243
:1034B0008E4BFCF759FF8046FDF770F88C49086089
:1034C0000846006801F07AFA8948006801F038FB84
:1034D00002F056FF8748006801F038FA002086495C
:1034E00008604FF07E50854908600620FFF708FE0F
:1034F000F8B1834801F0A6FE68480079674A52791E
:1035000010FB02F000EB8000400000EB4002C2EB39
:10351000C010624A127A694B53F8222002EBC001B4
:10352000012002F085FB01207649087000207249D5
:1035300008600520FFF7E4FDB0B158480079574A0C
:10354000527910FB02F000EB8000400000EB4002DB
:10355000C2EBC010514A127A584B53F8222002EBAA
:10356000C001002002F064FB0820FFF7C9FDD8B1BC
:103570004A4991F9060002F0ADFB48480079474AF4
:10358000527910FB02F000EB8000400000EB40029B
:10359000C2EBC010414A127A484B53F8222002EB8A
:1035A000C001022002F044FB0B20FFF7A9FD002818
:1035B00070D00B20544908730846027B53A10D308C
:1035C000FCF7D2FD5448007800F00F0030304E492F
:1035D0000A7B0D3188544C48007B401C0D39087320
:1035E00000214948027B0D30815401F0D7FC4A4844
:1035F0000068FCF79AFF804648480068FCF795FF92
:1036000081464146FCF772FE07464549FCF73CFE01
:1036100006464449FCF738FE0546FCF798FF044689
:103620003D480168204601F0EDFC374802F05EFBA2
:103630000D20FFF70DFD3C48007802282AD13648BE
:103640000068401C344908603848006828B1374891
:10365000006840F2DC51884206D940F2DC52002179
:103660000B2002F087FC0CE03048006800EB800083
:1036700080000A21B0FBF1F4224600210B2002F069
:1036800079FC00202A4908602A48007818B94FF0D0
:10369000FF3051E062E05EE0000230003C060020B6
:1036A00086000020691F0008CD1C0008ED5E0008A0
:1036B00014650008E960000836000020E86400088E
:1036C000F864000856474B6974426F6172645F3258
:1036D000323132530000000092000020040000202C
:1036E00000000020000048420000E03F00408F4002
:1036F0000C0000201C0000201400002010000020FE
:10370000C1510008080000202C05002068656C6C81
:103710006F20776F726C640020000020240000206E
:103720000000C84200002041350000202C0000208D
:10373000280000203400002001F040FC964800687A
:10374000401C95490860084600680A2803D10020FB
:103750000860924908600020914908700C20FFF72A
:10376000CFFC20B102F03AFA00208E4908600A200E
:10377000FFF7C6FC00287DD08B480068401C8A49B2
:1037800008608A49B1F9080001F0BAF98648006872
:1037900001F0A0F900218548153001F0EBF9002176
:1037A0008248153001F024F97E480068FCF7CFFE0E
:1037B00084B22146002001F0E5F87C48017D1530F7
:1037C00002F04AFB4FF4807178481530FCF7E5FCB5
:1037D00077480078022852D17648006801F0EEFB65
:1037E0007249B1F9080001F0B9FB73480068FCF7B1
:1037F0009CFE80466C480068FCF797FE8146414677
:10380000FCF774FD07466D49FCF73EFD06466C4922
:10381000FCF73AFD0546FCF79AFE04466648016847
:10382000204601F0EFFB6348006828B1614800685A
:1038300040F2DC51884206D340F2DC5200210B20DA
:1038400002F098FB0CE05B48006800EB8000800011
:103850000A21B0FBF1F4224600210B2002F08AFB82
:1038600001204F49087000204B490860514800680A
:103870004A4900E00EE0086000204E4908604C48CC
:103880000078032804D1002211460B2002F072FBBD
:10389000FDF7F6FC0E20FFF733FC08B102F09EF9AD
:1038A0000720FFF72DFC38B100204649087002F0D0
:1038B00077F80B20FFF7CCFB0320FFF721FCE8B3E0
:1038C00041480078D0B300203F4908703A4800686A
:1038D000401C394908603C4890F800013B49087396
:1038E0000846007BB0F5807F01DD00200873374873
:1038F000027B3549491C0D30FCF736FC33480D304E
:1039000001F04CFB2C480068FCF70FFE804626486F
:103910000068FCF70AFE81464146FCF7E7FC0746D3
:103920002649FCF7B1FC06462549FCF7ADFC0546E7
:10393000FCF70DFE04462048016800E005E0204643
:1039400001F060FB214802F0D1F90220FFF7D8FB1B
:1039500060B11F48007848B100201D490870A1F8E7
:10396000000100211A48401C01F068F80920FFF707
:10397000C7FB48B10A211748FFF78DFA154988722D
:103980000B21144801F006FCFFF7E4FB1249087014
:1039900002F0D6F868E50000300000202C0000207E
:1039A0003400002014000020240000201404002013
:1039B0003500002028000020200000200000C84220
:1039C0000000204108000020100200202C050020EB
:1039D000120300203C0600200400002070B50446BD
:1039E0000723012221460A48FDF768F8012108480B
:1039F000FDF7C5F800BF02210548FDF724F80028AF
:103A0000F9D00348FDF71BF80546284670BD0000B5
:103A1000002401402DE9FF5F1120FFF7DFFF029036
:103A20000120FFF7DBFF03900298FCF783FD0446BB
:103A30000D460398FCF779FD0090FCF79CFD80464D
:103A40004FF03332074BFCF78FFC064622462B46DD
:103A5000FCF7FCFC8246FCF7A1FD0190019804B044
:103A6000BDE8F09F3333F33F08B501214802FDF76D
:103A7000D1FC0220ADF8000000208DF8030069465B
:103A80001D48FDF753FA00201C4908600871487171
:103A90004FF4602088600020C86001200874184836
:103AA000FCF7E4FF0523012211461548FDF706F84F
:103AB0000523022211211248FDF700F801211048C8
:103AC000FCF7A8FF0120FDF76BF80D48FDF752F851
:103AD00000BF0B48FCF7C0FF0028FAD10848FDF7EB
:103AE00059F800BF0648FCF7A0FF0028FAD10121D1
:103AF0000348FDF744F808BD0008014048070020CE
:103B00000024014070B50446FB4890F90000401EB7
:103B1000C0EBC00101EB4010F84951F8200000282B
:103B20007ED0F54890F90000401EC0EBC00101EBCB
:103B30004010F24901EB80008E30EF4991F90010FE
:103B4000491EC1EBC10202EB4111EC4A02EB8101BB
:103B50004968405C00287CD0002C7BD0E64890F976
:103B60000000401EC0EBC00101EB4010114601EB0C
:103B700080004030E04991F90010491EC1EBC102BC
:103B800002EB4111DD4A02EB8101496850F8211036
:103B9000491CD94890F90000401EC0EBC00202EB5E
:103BA0004010D64A02EB80004030D34A92F9002000
:103BB000521EC2EBC20303EB4212D04B03EB820254
:103BC000526840F82210CC4890F90000401EC0EB2B
:103BD000C00101EB4010194601EB80004030C6499E
:103BE00091F90010491EC1EBC10202EB41111A46C6
:103BF00002EB8101496850F82120BF4890F900008C
:103C0000401EC0EBC00101EB4010194601EB8000E3
:103C10007030B94991F90010491EC1EBC10300E0B1
:103C2000D9E103EB4111B54B03EB8101496850F831
:103C30002100824236DBB04890F90000401EC0EB04
:103C4000C00101EB4010194601EB80005830AA4931
:103C500001E012E127E091F90010491EC1EBC10219
:103C600002EB41111A4602EB8101496850F821200C
:103C7000A14890F90000401EC0EBC00101EB4010CC
:103C8000194601EB800040309B4991F90010491E14
:103C9000C1EBC10303EB4111984B03EB8101496870
:103CA00040F821209FE0944890F90000401EC0EBAE
:103CB000C00101EB4010914901EB800040308E497A
:103CC00091F90010491EC1EBC10202EB41118B4A70
:103CD00002EB8101496850F82110491E864890F98D
:103CE0000000401EC0EBC00202EB4010834A02EB12
:103CF00080004030804A92F90020521EC2EBC2037D
:103D000003EB42127D4B03EB8202526840F8221013
:103D1000794890F90000401EC0EBC00101EB401053
:103D2000194601EB80004030734991F90010491E9B
:103D3000C1EBC10202EB41111A4602EB8101496855
:103D400050F821206C4890F90000401EC0EBC001E3
:103D500001EB4010194601EB80005830664991F99B
:103D60000010491EC1EBC10303EB4111634B03EB90
:103D70008101496850F82100824234DA5E4890F9A6
:103D80000000401EC0EBC00101EB4010194601EBE2
:103D900080007030584991F90010491EC1EBC102F2
:103DA00002EB41111A4602EB8101496850F82110DB
:103DB000491E514890F90000401EC0EBC00202EBC2
:103DC00040101A4602EB800040304B4A92F9002026
:103DD000521EC2EBC20303EB4212484B03EB8202BA
:103DE000526840F8221046480068002844D04248F3
:103DF00090F90000401EC0EBC00505EB40103F4DA0
:103E000005EB800040303C4D95F900506D1EC5EB30
:103E1000C50606EB4515394E06EB85056D6850F86D
:103E20002530354890F90000401EC0EBC00505EB79
:103E30004010354605EB80008E302F4D95F900502F
:103E40006D1EC5EBC50606EB45152C4E06EB85052C
:103E50006D68425D284890F90000401EC0EBC00527
:103E600005EB4010354605EB80004168224890F98B
:103E70000000234D2D68A84787E0E4B31E4890F961
:103E80000000401EC0EBC00101EB40101B4901EBDC
:103E900080004068401E184991F90010491EC1EB8E
:103EA000C10202EB4111154A02EB81014860124840
:103EB00090F90000401EC0EBC00101EB401011461C
:103EC00001EB8000406800285FDA0B4890F90000A1
:103ED000401EC0EBC00101EB4010114651F820001C
:103EE000401E054991F90010491EC1EBC10202EBC9
:103EF0004111024A06E009E0B50100201C11002032
:103F0000BC01002002EB810148603EE0324890F99C
:103F10000000401EC0EBC00101EB40102F4901EB37
:103F200080004068401C2C4991F90010491EC1EBEB
:103F3000C10202EB4111294A02EB81014860264887
:103F400090F90000401EC0EBC00101EB401011468B
:103F500001EB80004168204890F90000401EC0EB52
:103F6000C00202EB40101D4A52F8200081420CDBD7
:103F70000021194890F90000401EC0EBC00202EB7E
:103F80004010164A02EB80004160134B93F9003059
:103F90005B1EC3EBC30505EB4313104D05EB830319
:103FA00003F140010C4B93F900305B1EC3EBC305DA
:103FB00005EB4313094D05EB83035868064B93F952
:103FC00000305B1EC3EBC30505EB4313034D05EB4C
:103FD00083039A68904770BDB50100201C11002032
:103FE0002DE9F0410446002C7ED1EA4890F900000A
:103FF000401EC0EBC00101EB4010E74901EB80001F
:104000008830E44991F90010491EC1EBC10202EB6E
:104010004111E14A02EB81014968405C01287CD1F1
:10402000DC4890F90000401EC0EBC00101EB4010DD
:10403000114601EB80008E30D64991F90010491EDF
:10404000C1EBC10202EB4111D34A02EB8101496885
:10405000405C08B9012200E00022CE4890F900003F
:10406000401EC0EBC00101EB4010CB4901EB8001C9
:104070008E31C84890F90000401EC0EBC00303EB2E
:104080004010C54B03EB800040680A54C14B93F9C4
:1040900000305B1EC3EBC30505EB4313BE4D05EBC0
:1040A000830303F14001BB4B93F900305B1EC3EB6C
:1040B000C30505EB4313B84D05EB83035868B54BB7
:1040C00093F900305B1EC3EBC30505EB4313B24D00
:1040D00005EB83039A689047B0480068E8B1AD4D9E
:1040E00095F900506D1E00E0A9E0C5EBC50606EB92
:1040F0004515A94E06EB85054035A64E96F900609C
:10410000761EC6EBC60707EB4616A34F07EB8606DF
:10411000766855F826309F4D00E032E095F9005062
:104120006D1EC5EBC50606EB45153E4606EB85053F
:104130008E35984E96F90060761EC6EBC60707EBE3
:104140004616954F07EB86067668AA5D914D95F960
:1041500000506D1EC5EBC50606EB45153E4606EB49
:10416000850569688B4D95F900506D1EC5EBC50638
:1041700006EB45153E4606EB8505E868874D2D683C
:10418000A847844890F90000401EC0EBC00101EB35
:104190004010814901EB800088307E4991F9001080
:1041A000491EC1EBC10202EB41117B4A02EB8101C6
:1041B0004968405C022842D1764890F90000401ED0
:1041C000C0EBC00101EB4010114601EB800028302C
:1041D000704991F90010491EC1EBC10202EB411177
:1041E0006D4A02EB8101496810F8210040B269492B
:1041F00008700B4693F900305B1EC3EBC30505EB5B
:104200004313154605EB830303F14001614B93F91A
:1042100000305B1EC3EBC30505EB4313154605EBEE
:10422000830358685B4B93F900305B1EC3EBC305F7
:1042300005EB4313154605EB83039A689047012C61
:104240007ED1544890F90000401EC0EBC00101EB44
:104250004010514901EB80000069002870D04D48A2
:1042600090F90000401EC0EBC00101EB40104A492C
:1042700001EB8000002140F88E1F818047480068D4
:10428000F0B3444D95F900506D1EC5EBC50606EB25
:104290004515414E06EB850540353E4E96F90060CA
:1042A000761EC6EBC60707EB46163B4F07EB8606A6
:1042B000766855F82630374D95F900506D1EC5EBE0
:1042C000C50606EB45153E4606EB85058E35314E97
:1042D00096F90060761EC6EBC60707EB46162E4F12
:1042E00007EB86067668AA5D2A4D95F900506D1E8B
:1042F000C5EBC50606EB45153E4606EB850500E019
:104300000FE06968234D95F900506D1EC5EBC50699
:1043100006EB45153E4606EB8505E8681F4D2D6802
:10432000A8471C4890F90000401EC0EBC00101EBFB
:104330004010194901EB8000007C40B2154900E0B3
:1043400026E008700B4693F900305B1EC3EBC305F3
:1043500005EB4313104D05EB830303F140010D4BB7
:1043600093F900305B1EC3EBC30505EB43130A4D05
:1043700005EB83035868074B93F900305B1EC3EBD2
:10438000C30505EB4313044D05EB83039A6890477F
:10439000BDE8F081B50100201C110020BC01002007
:1043A00010B5044601F036F901207649C860764818
:1043B0008860002008610220886281F8880001205E
:1043C00081F88E00002048600220086002216D48BC
:1043D000C0F8A8106D49C0F8A4100021C0F8AC10B6
:1043E0000321C0F8C410022180F824110421C0F870
:1043F000C810022180F825110521C0F8CC10022137
:1044000080F826110621C0F8D010022180F827116B
:104410000721C0F8D410022180F828110021C0F82B
:10442000A01005205749C1F89C0003215548C0F849
:1044300044115749C0F840110221C0F84811002129
:10444000C0F86011012180F8C011002180F8C61168
:10445000C0F83C1100204B49C1F8380107214948F8
:10446000C0F8B4134B49C0F8B0130221C0F8B81318
:104470000021C0F8D01300204249C1F8A80304214C
:104480004048C0F8E0114449C0F8DC110221C0F8EE
:10449000E4110021C0F8FC11012180F85C12002118
:1044A00080F86212C0F8D81100203649C1F8D40152
:1044B00005213448C0F87C123849C0F8781202212E
:1044C000C0F88012012180F8F812002180F8FE1255
:1044D000012180F8F912002180F8FF12012180F8F3
:1044E000FA12002180F80013C0F874120320254945
:1044F000C1F8700206212348C0F818132849C0F8F3
:1045000014130221C0F81C13012180F89413042114
:10451000C0F87C13012180F895132021C0F8801386
:10452000012180F89613C821C0F88413012180F876
:1045300097136FF00801C0F870131521C0F88813A5
:10454000012180F89813C0F870130721C0F88C136C
:104550000021C0F8101305200A49C1F80C031148C6
:104560000460114890F90000401EC0EBC00101EB4F
:104570004010044901EB8000002182680846904702
:1045800010BD00001C110020814600085950000891
:10459000D94E0008E1450008014C0008ED4700082D
:1045A000854C0008BC010020B501002010B5054C69
:1045B00044F82010183444F82020183444F82030EF
:1045C00010BD000068140020014908607047000019
:1045D000DC0100200149087070470000D80100206C
:1045E000F8B505460E4619480078062829D000F08F
:1045F00051FF002404E02146012000F09CFF641CD0
:104600000C2CF8DD12A301224FF48171002001F07F
:1046100001F91148006811A302220A21009000202C
:1046200001F0F8F80F4800780FA303220A21009048
:10463000002001F0EFF80FA304220A21002001F06E
:10464000E9F8062001490870F8BD0000B401002017
:10465000496E666F72000000DC01002054503A2061
:1046600025730000D80100205645523A20562530C7
:10467000327800004D443A20564F4C4C474F0000D2
:1046800070B504460D461948007800281ED018A3BE
:104690000B220A21012000F027FE002301221146EF
:1046A000184600F05BFF18A301225021002001F002
:1046B000B1F819A302225F21002001F0ABF819A381
:1046C00003225F21002001F0A5F80AE00CB90121C6
:1046D00000E00021084615A3052240F2031101F075
:1046E00099F800200149087070BD0000B401002055
:1046F000C9EEDBDACAD0CED6BDF8BFC6BCBCD3D0BB
:10470000CFDEB9ABCBBE000056472D2D2D2D2D2D64
:104710002D2D2D2D2D2D0000467265712E2A2A2A51
:10472000000000005077722E2A2A0000454E5445A2
:104730005200000010B504462346012250210020FB
:1047400001F068F810BD00002DE9FC410446204648
:10475000FBF7EBFE80460849FBF7C8FD0546FBF773
:104760000AFF06A30222CDE900015021002001F03A
:1047700051F8BDE8FC81000000247449467265715F
:104780002E25362E32664D487A0000002DE9FC4178
:1047900004462046FBF7C9FE80460849FBF7A6FD04
:1047A0000546FBF7E8FE06A30422CDE900015F21E0
:1047B000002001F02FF8BDE8FC81000000007A44E1
:1047C00042722E252E33666B6200000038B5044617
:1047D00003A303225F210020009401F01BF838BDE1
:1047E0005077722E256464426D00000070B5044657
:1047F0000E4623480078042817D000F04BFE002511
:1048000004E02946012000F096FE6D1C0C2DF8DD19
:104810001CA301224FF48171002000F0FBFF00F087
:1048200061F800F03DF800F07FF8042014490870AA
:1048300008460078042821D10CB9012100E00021AC
:10484000084613A302224FF4817100F0E3FF012C0C
:1048500001D1012100E0002108460EA303224FF4FC
:10486000817100F0D7FF022C01D1012100E000216D
:10487000084609A30222712100F0CCFF70BD0000A0
:10488000B4010020436F6E74696E756F757300001C
:10489000545800005258000054585F4D4400000026
:1048A0002DE9FC410A480068FBF73FFE074609492D
:1048B000FBF71CFD0446FBF75EFE07A30322CDE9D0
:1048C000000140F20311002000F0A4FFBDE8FC81CC
:1048D000C401002000007A4425372E33666B6270D5
:1048E000730000002DE9FC410A480068FBF71DFE3B
:1048F00007460949FBF7FAFC0446FBF73CFE07A311
:104900000222CDE900010521002000F083FFBDE86F
:10491000FC810000CC0100200024744925362E3291
:10492000664D487A0000000008B5054890F900007F
:1049300004A3032205210090002000F06BFF08BDB6
:10494000D0010020256464426D0000007CB504465F
:104950000748007804280AD12046FBF70CFE05A37F
:104960000522CDE900010A21002000F053FF7CBDA3
:10497000B4010020726174653D25362E326625250E
:1049800000000000FEB505460C46084800780428E3
:104990000BD12846FBF7EFFD05A304228DE8130099
:1049A00040F20311002000F035FFFEBDB4010020ED
:1049B00025352E3166252520253464007CB5044636
:1049C0000748007804280AD12046FBF7D4FD05A348
:1049D0000422CDE900010A21002000F01BFF7CBD6C
:1049E000B4010020433D25362E32666D41000000A3
:1049F000F8B504460D4600260C480078042814D16A
:104A000029462046FEF72EFC09480AA3052212215A
:104A10000090002000F0FEFE0548143005A3062299
:104A200012210090002000F0F5FEF8BDB401002036
:104A300060150020252D313573000000F8B50446BF
:104A40000D46002614480078032823D113A305221D
:104A50000A21002000F0DEFEADB117A305220A21D5
:104A6000002000F0D7FE00BF0AE0207806F10C021B
:104A700013A30A210090002000F0CCFE641C761CD9
:104A8000AE42F2DB06E00FA305220A2100200094CB
:104A900000F0C0FEF8BD0000B4010020202020205E
:104AA0002020202020202020202020202020202006
:104AB00020202020000000007061636B65743D00C1
:104AC000257800007061636B65743D252D31357369
:104AD0000000000038B5044606480078032807D1D6
:104AE00005A303224FF481710020009400F092FE90
:104AF00038BD0000B40100202530366400000000FD
:104B000038B504460B480078032812D114F1960FEB
:104B10000FDD0A2C0DDA42F2107094FBF0F100FB6D
:104B2000114505A3022240F203110020009500F078
:104B300071FE38BDB40100202530346464426D003C
:104B40007CB504460748007803280AD12046FBF7C5
:104B500012FD05A30222CDE900010521002000F08D
:104B600059FE7CBDB4010020252D362E32666D41E4
:104B700000000000F8B504460D4600261B480078EA
:104B8000032831D195B100BF0AE0207806F10A016F
:104B900017A305220090002000F03CFE641C761C48
:104BA000AE42F2DB29462046FEF73EFB2946204670
:104BB000FEF73AFB0F4810A30422122100900020B8
:104BC00000F028FE0B4814300BA3052212210090A0
:104BD000002000F01FFE0748283007A306221221FC
:104BE0000090002000F016FEF8BD0000B401002087
:104BF0002578000060150020252D31357300000058
:104C000070B505460E4617480078032817D000F007
:104C100041FC002404E02146012000F08CFC641CCF
:104C20000C2CF8DD10A301224FF48171002000F05C
:104C3000F1FD10A303220521002000F0EBFD03206D
:104C4000084908700846007803280AD10DB90121E7
:104C500000E00021084609A3062240F2031100F0FB
:104C6000D9FD70BDB40100205061636B65742052A2
:104C7000580000005061636B65743A005354415210
:104C8000540000002DE9FF4704460E465B480078BB
:104C900005282FD000F0FEFB002504E02946012066
:104CA00000F049FC6D1C0C2DF8DD55A301224FF4DA
:104CB0008171002000F0AEFD53A302220A210020E2
:104CC00000F0A8FD52A303220A21002000F0A2FD5B
:104CD00054A304220A21002000F09CFD55A30522C4
:104CE0000A21002000F096FD56A306220A2100208A
:104CF00000F090FD0520414908700846007805281D
:104D000079D155480068082202EB820202F10A01BB
:104D100000900CB9012200E0002210464FA30222AD
:104D200000F078FD4E480068FBF7FFFB82464D49D6
:104D3000FBF7DCFA8146FBF71EFCCDE90201706847
:104D4000082202EB820202F10A010090012C01D13B
:104D5000012200E00022104643A3032200F05AFD86
:104D600044480068FBF7E1FB82463E49FBF7BEFA88
:104D70008146FBF700FC082202EB8202CDE900012C
:104D800002F10A01022C01D1012200E000221046AA
:104D900039A3042200F03EFD394890F900000A22B0
:104DA000082302EBC3010090032C01D1012200E093
:104DB0000022104633A3052200F02CFD3348006882
:104DC000FBF7B3FB82463249FBF790FA8146FBF7CB
:104DD000D2FB082202EB8202CDE9000102F10A01B6
:104DE000042C02D1012201E005E00022104629A393
:104DF000062200F00FFDBDE8FF870000B40100208F
:104E000053657474696E6700547970653A000000E8
:104E100043686E6C3A2D2D2D2D2D2D2D2D2D2D4DC4
:104E2000487A0000537465703A2D2D2D2D4D487A27
:104E3000000000005478506F7765723A2D2D2D6474
:104E4000426D0000526642723A2D2D2D2E2D2D2DD1
:104E50006B62707300000000D40100202573000015
:104E6000CC01002000247449253032642D3E2536C3
:104E70002E326600C801002025342E326600000064
:104E8000D00100202530336400000000C401002060
:104E900000007A4425372E3366000000014908607F
:104EA00070470000C80100200149086070470000F9
:104EB000CC0100200149086070470000C4010020B7
:104EC0000149087070470000D001002001490860C6
:104ED00070470000D401002070B505460E46174803
:104EE0000078022817D000F0D5FA002404E021460B
:104EF000012000F020FB641C0C2CF8DD10A3012223
:104F00004FF48171002000F085FC10A302220521DE
:104F1000002000F07FFC0220084908700846007855
:104F200002280AD10DB9012100E00021084609A399
:104F3000062240F2031100F06DFC70BDB4010020A8
:104F40005061636B65742054580000005061636BBE
:104F500065743A00535441525400000038B5044679
:104F60000B480078022812D114F1960F0FDD0A2C9D
:104F70000DDA42F2107094FBF0F100FB114505A32D
:104F8000032240F203110020009500F043FC38BDDD
:104F9000B40100202530346464426D0010B504462D
:104FA00005480078022805D1234603220A21002063
:104FB00000F030FC10BD0000B401002038B50446FC
:104FC0000B480078022811D1601C38B909A30122CE
:104FD00040F20311002000F01DFC07E007A30122AE
:104FE00040F203110020009400F014FC38BD0000D2
:104FF000B40100202020204F555400002535646D59
:10500000730000002DE9FE4305460C460C4800786D
:10501000022812D12846FBF788FA81460949FBF796
:1050200065F90646FBF7A7FA07A302228DE81300ED
:1050300040F20311002000F0EDFBBDE8FE8300000C
:10504000B40100200000204125352E3166252520A1
:10505000202025356400000070B504460E4600F09F
:1050600019FA002504E02946012000F064FA6D1CBD
:105070000C2DF8DD01201C4908700CB9012100E05D
:105080000021084619A301220A2100F0C3FB012CCC
:1050900001D1012100E00021084619A302220A21C2
:1050A00000F0B8FB022C01D1012100E000210846EC
:1050B00018A303220A2100F0ADFB032C01D101212A
:1050C00000E00021084618A304220A2100F0A2FBF8
:1050D000042C01D1012100E00021084617A305227C
:1050E0000A2100F097FB70BDB4010020456E746585
:1050F00072205246205472616E736D69746572003D
:10510000456E746572205246205265636569766506
:1051100072000000456E74657220524620436F6E27
:1051200074696E756F757300456E746572205246B2
:105130002053657474696E6700000000456E7465E5
:10514000722044657669636520496E666F7200005F
:105150002DE9F04106460C460D4FB046204604EBC3
:10516000D0714910A4EB410109B1611C00E0214656
:105170008CB2002507E03846FCF7B9FA28F815008C
:10518000BF1C681C85B2A542F5DBBDE8F0810000BC
:1051900000E0030870B505460C46264604EBD670C1
:1051A0004010A4EB400008B1601C00E0204682B231
:1051B00029460248FCF79EFA70BD000000E0030893
:1051C0002DE9F0410746884614461848046040F629
:1051D000C410844202D9A4F6C41002E040F6C41000
:1051E000001B054612480078E8B14FF07E51114887
:1051F0000068FAF7F1FF0F490860C82D07D24FF099
:105200007E510D480068FAF7E7FF0B49086009482E
:10521000016809480068FBF769F806460749FBF78B
:1052200033F807490860BDE8F0810000180000204D
:105230000800002010000020140000200000C842D8
:105240001C00002010B586B00446224822490860A0
:105250000846FCF723FD0220ADF8040048208DF835
:10526000070002208DF8060001A91C48FBF75EFE2E
:1052700001210220FCF7BEF81D208DF8140000204B
:105280008DF8150001208DF816008DF8170005A87F
:10529000FCF740F80C20ADF808000220ADF80A0039
:1052A0000120ADF80C000020ADF80E00ADF81000A4
:1052B00002A90B48FCF77AFD01210948FCF755FDCE
:1052C000012210210648FCF7C7FD0648046006B01D
:1052D00010BD0000E15F000840010020000C01400B
:1052E000000400402C0100202DE9F05F81468A4631
:1052F00093461E46002569E000244FF0010812E0A5
:105300003548005D715D88420BD13349601C095CF2
:10531000681C305C814204D14FF6FF7000EA04182B
:1053200005E0A01C84B22C48005D7E28E8DC00BFAC
:10533000B8F1010F28D0022310225946504600F040
:10534000D4F800271BE0002415E0B9F1010F07D1C4
:10535000224911F80810C943C8B200F0E7FA04E086
:105360001E4911F8080000F0E1FA08F101001FFAE7
:1053700080F8601C84B2102CE7DB781C87B2022F07
:10538000E1DBA81C85B21DE00223102259465046DD
:1053900000F0ABF8002711E000240BE0B9F1010F99
:1053A00003D1FF2000F0C2FA02E0002000F0BEFAB4
:1053B000601C84B2102CF1DB781C87B2022FEBDB6F
:1053C000681C85B20AF1100000F0FF0A705D002829
:1053D00092D1BDE8F09F00001D6500083E65000801
:1053E0002DE9FF5F0C4615461E460027AA4648E0F9
:1053F000F05D202843DBF05D7E2840DCF05D203846
:105400001FFA80F90120C0EB450102230822204643
:1054100000F06BF8A346AA464FF0000827E0B8F169
:10542000080F02D10AF1010AA3460BF1010BBAF1F0
:105430000C0F00DD1EE0BBF1C00F00DD1AE000988C
:10544000012809D1124901EB091111F80810C943CB
:10545000C8B200F06BFA06E00D4901EB091111F832
:10546000080000F063FA08F101001FFA80F8B8F1B3
:10547000100FD4DB00BF0834C02C00DD04E0781C22
:1054800087B2F05D0028B3DC00BFBDE8FF9F0000DD
:105490003E67000810B50C23C0220121084600F029
:1054A00024F8002403E0002000F040FA641CB4F566
:1054B000106FF8DB10BD0022002100BF06E00022C3
:1054C00001E0531C9AB20A2AFBDB491C8142F6D345
:1054D000704710B50446302000F056F9F02000F077
:1054E00011FA204600F022FA10BD2DE9F0410446E1
:1054F0000D4616461F46641EED1D302000F044F98F
:10550000152000F0FFF9E0B200F010FAA119491ED1
:10551000C8B200F00BFA752000F0F4F9E8B200F020
:1055200005FAE919491EC8B200F000FA5C2000F043
:10553000E9F9BDE8F08170B505460E460123082261
:1055400031462846FFF7D1FF002403E0FF2000F09A
:10555000EDF9641C042CF9DB70BD00002DE9F05F4F
:1055600007460D4616461C46A946B246284800EB9B
:10557000C400B0F802B04FEAEB700BEB5070C310F0
:10558000234830F8342031462846FFF7AEFF4FF06D
:1055900000082BE009F10109B9F1C00F03DDA946AC
:1055A0000AF1010A20E0BAF10C0F00DD2DE0012F15
:1055B00009D1174901EBC40149680978C943C8B248
:1055C00000F0B4F906E0124901EBC401496808781B
:1055D00000F0ACF90E4800EBC4004068401C0C49D8
:1055E00001EBC401486000BF08F10108084931F827
:1055F0003410074A02EBC402528801FB02F0C117C3
:1056000000EB5171B8EBE10FC4DB00BFBDE8F09FC8
:10561000740F002008B51020ADF800008DF80300CD
:1056200003208DF8020069465448FBF77FFC802078
:10563000ADF8000010208DF8030003208DF8020063
:1056400069464E48FBF772FC4020ADF80000102080
:105650008DF8030003208DF8020069464748FBF7E8
:1056600065FC2020ADF8000010208DF80300032019
:105670008DF8020069464148FBF758FC01221021D1
:105680003E48FBF739FD002220213C48FBF734FD62
:105690006420FFF710FF012220213848FBF72CFD82
:1056A00042F21070FFF707FF302000F06DF89420F1
:1056B00000F028F9312000F067F8D72000F022F937
:1056C0009F2000F033F9322000F01CF9002000F098
:1056D0002DF9012000F02AF9032000F027F93020ED
:1056E00000F052F8082000F00DF9752000F00AF9DA
:1056F000002000F01BF9142000F018F9152000F02C
:1057000001F9002000F012F9FF2000F00FF9BC2091
:1057100000F0F8F8002000F009F9A62000F006F9E2
:10572000CA2000F0EFF8002000F000F99F2000F000
:10573000FDF8202000F0FAF81020FFF7CAFEFA204A
:1057400000F02EF8202000F0DDF80B2000F0EEF83D
:1057500042F21070FFF7AFFEAF2000F0D3F842F234
:105760001070FFF7A8FEFFF795FE05480549486051
:105770005E2008804820488008BD0000000C0140E1
:10578000CE6D0008740F002010B504460348007861
:10579000A04202D0204600F0B5F810BD8F010020D5
:1057A00010B50446C4F30804302000F0ABF88120A3
:1057B00000F0A8F804F03F0000F0B8F8A00900F0ED
:1057C000B5F810BD10B5012240210748FBF794FC45
:1057D000012280210448FBF78FFC0022802102482F
:1057E000FBF78AFC10BD0000000C014010B501223F
:1057F00040210748FBF780FC002280210448FBF78A
:105800007BFC012280210248FBF776FC10BD0000E2
:10581000000C01400FB4F0B58FB006460C46174699
:1058200018A80E90342101A8FAF7B7FC322101A87C
:105830000E9B179AFCF758FD01A8FAF7B9FC05462C
:10584000C02D00DDC025B4F5817F06D101A8FAF78F
:10585000AFFCC0004508C5F1600440F2031084426B
:1058600005D101A8FAF7A4FCC500C5F1C00440F2B7
:105870000110844200D1012401AB3A462146304652
:10588000FFF7AEFD00200E900FB0F0BC5DF814FBEA
:1058900070B50446002520E0002240211848FBF79F
:1058A0002BFC04F0800028B1012280211448FBF772
:1058B00023FC04E0002280211148FBF71DFC01229B
:1058C00040210F48FBF718FC002240210C48FBF751
:1058D00013FC6006040E681CC5B2082DDCDB002238
:1058E00080210748FBF708FC012240210448FBF710
:1058F00003FC002240210248FBF7FEFB70BD0000C4
:10590000000C014010B5044607480470FFF75AFF29
:105910007820FFF7BDFF8020FFF7BAFF2046FFF792
:10592000B7FFFFF763FF10BD8F01002010B50446DD
:10593000FFF748FF7820FFF7ABFFC020FFF7A8FF75
:105940002046FFF7A5FFFFF751FF10BD70B50546D4
:10595000002605E0601CC4B2C82C01DD002070BD2B
:1059600002210E48FBF786FE0028F3D029460B489B
:10597000FBF78CFE002405E0601CC4B2C82C01DDDE
:105980000020ECE701210548FBF774FE0028F3D066
:105990000248FBF778FEC6B23046E0E7003001402F
:1059A00010B50648006800B910BD00200449087011
:1059B0003620FBF7AFFF00BFF6E70000FC01002038
:1059C000000200200121014A1170704702020020EC
:1059D00010B586B0044601210803FBF71BFDE0204B
:1059E000ADF8140018208DF8170003208DF816006C
:1059F00005A92348FBF79AFA0020ADF800004FF400
:105A00008270ADF802000020ADF80400ADF8060089
:105A1000ADF808004FF40070ADF80A001820ADF89A
:105A20000C000020ADF80E000720ADF8100069460C
:105A30001448FBF72DFE01211248FBF70FFE102042
:105A4000ADF814008DF8170003208DF8160005A995
:105A50000B48FBF76BFA0220ADF8140048208DF8D4
:105A6000170003208DF8160005A90748FBF75EFA1A
:105A7000FBF7A8F800F00CF80448046006B010BD6D
:105A80000008014000300140000C014004020020E9
:105A90001FB50220ADF8000003208DF80200482059
:105AA0008DF8030069461748FBF740FA0220FBF720
:105AB00011F90220019000208DF8080008208DF8CF
:105AC000090001208DF80A0001A8FBF71DF901214A
:105AD0000846FBF70BFA07208DF80C0001208DF823
:105AE0000D0000208DF80E0001208DF80F0003A896
:105AF000FBF710FC0448054908600846FBF7D2F89C
:105B00001FBD0000000C0140D15E0008080200200B
:105B100070B505460C460748FFF75AFFFBF778FDBE
:105B20003420FBF7F7FE0CB103480460E52003497D
:105B3000086070BDC5590008F8010020FC01002074
:105B400010B5ADF50A7D2148006810B90DF50A7D44
:105B500010BD1F48007800B9F8E700201C49087004
:105B60001C480078012802D002282BD11AE02021FD
:105B70000DF22510FBF716FD3420FBF7CBFE0020BD
:105B80001449087020208DF824014FF4867247A92B
:105B90006846FAF7E9FA00200F4C44A90EC92468B8
:105BA000A04710E000200B4908704FF4867247A907
:105BB0006846FAF7D9FA0320074C44A90EC92468AD
:105BC000A04700E000BF00BF00BFBFE7FC0100200E
:105BD0000202002000020020F801002010B5094850
:105BE000006800B910BD0120074908703620FBF796
:105BF00091FE3A20FBF78EFE3420FBF78BFE00BFB0
:105C0000F0E70000FC0100200002002003490968C1
:105C100001B970470249086000BFFAE7FC010020A3
:105C2000F4010020014908707047000001020020C3
:105C300070B504460D461B48006800B970BD0021D0
:105C40000846FFF765FF1848006800F031F824B1F6
:105C5000012C14D0022C21D110E00420134908702B
:105C600033211220FCF72AFB3620FBF753FE3B20A2
:105C7000FBF750FE3520FBF74DFE10E00FE0032050
:105C80000A49087035210820FCF718FB0D21022075
:105C9000FCF714FB3420FBF73DFE00E000BF00BF23
:105CA00000BFCBE7FC010020F00100200002002033
:105CB00010B504460548006800B910BD04480460EA
:105CC00001780A20FCF7FAFA00BFF6E7FC01002091
:105CD000F00100200349096801B9704702490870C2
:105CE00000BFFAE7FC010020EC01002010B50446DB
:105CF0000648006800B910BD022005490870217BE4
:105D000004F10D00FBF77EFD00BFF4E7FC0100206D
:105D1000000200207FB505460C4619481949086065
:105D20000846FBF773FF0121C802FBF773FB19203C
:105D30008DF8000000208DF801008DF80200012090
:105D40008DF803006846FBF7E5FAA8B2ADF8080045
:105D50004720ADF804000020ADF80A00ADF80600B9
:105D600001A90948FCF7AEF8012211460648FCF7E4
:105D700073F801210448FBF7F8FF044804607FBD75
:105D8000C95F000898010020002C01409401002008
:105D900030B587B005460C462A482B4908600846AE
:105DA000FCF748F901218803FBF734FB4FF400703E
:105DB000ADF8180003208DF81A0018208DF81B008C
:105DC00006A92248FBF7B2F84FF48060ADF818003E
:105DD00004208DF81B0006A91C48FBF7A7F8252016
:105DE0008DF8040003208DF805008DF806000120D1
:105DF0008DF8070001A8FBF78DFA02950020ADF899
:105E00000C00ADF80E00ADF81000ADF814000C2039
:105E1000ADF8120002A90E48FCF7B8F9012240F2D1
:105E200025510B48FCF78DF9012240F22441084826
:105E3000FCF787F901210648FCF740F905480460A2
:105E400007B030BD8D60000810010020000801403F
:105E5000003801400801002070B504460D4603E0FB
:105E6000207800F007F8641C281EA5F101018DB20E
:105E7000F6D170BD10B5044600BF40210448FCF7C0
:105E800029F90028F9D021460148FCF7F0F910BDA6
:105E90000038014010B501210420FBF7BBFA0121B5
:105EA0000820FBF7B7FA01211020FBF7B3FA012114
:105EB0002020FBF7AFFA01210803FBF7ABFA012121
:105EC0000846FBF7A7FA4FF48040FBF787FA10BDAE
:105ED00070B504460D460448006818B10120024917
:105EE0000968884770BD0000040200200FB410B597
:105EF00004464FF48C7203A91A48FAF735F934B105
:105F0000012C1CD0022C1ED0032C25D11FE0FFF742
:105F100065FE0A20FDF7CAF81348007870B1032225
:105F200012A110481530FAF74AF938B94FF07E51EE
:105F30000F480068FAF750F90D4908600DE00E208F
:105F4000FDF7B4F809E00E20FDF7B0F805E0FBF727
:105F500067F9FFF743FE00E000BF00BF10BC5DF82B
:105F600014FB0000140400200800002068656C0089
:105F70001400002070B504460E4615460120FCF7BB
:105F8000D8F904EB44000E4901EB80008560002045
:105F900004EB44010A4A02EB8101486004EB44002F
:105FA000114601F8206035B90120A0400549096873
:105FB0000843044908600020FCF7BBF970BD0000ED
:105FC0009C0F0020A801002070B504460D46034830
:105FD000006810B101480068804770BD940100203E
:105FE00070B504460D462148008840B92048FBF7AB
:105FF000C8FE2049088001201C49088034E01B4865
:106000000088012830D11A48FBF7BBFE1A490880E6
:106010000846008817490988884207DD1648008825
:1060200014490988401A1549086009E01148008898
:106030004FF6FF71081A1049098808440F49086093
:106040000F4800680D490968B0FBF1F00D49086080
:106050000020064908800B48026807480188054867
:106060000088094B1B68984770BD00002001002084
:10607000000400401C0100201E010020240100201B
:10608000F4000020280100202C01002070B50446F7
:106090000D4614B1012C1ED10DE0104801881048A6
:1060A000104A12689047FF210D48FAF776F8002051
:1060B0000A49088010E00A48084A128885540748AF
:1060C0000088401C0549088008460088FE2801DD3C
:1060D0000020088000E000BF00BF70BD0C01002060
:1060E00047060020080100202DE9F04107460D4633
:1060F00014461E46781E06287DD2DFE800F07C0399
:106100002B51046828E125B1012D10D0022D1ED19C
:1061100015E00CB1052100E006210846FCF7C6FF9A
:106120000CB1042000E000208D49087010E00CB193
:10613000062100E007210846FCF7B8FF08E00CB193
:10614000082100E007210846FCF7B0FF00E000BF8F
:1061500000BF01E115B1012D1ED11EE014B14FF4B5
:10616000FA7300E000231A460CB1012300E000237B
:1061700019460CB10B2300E007231846FFF7FAFE7F
:106180000CB1022000E0002075490870002075491C
:1061900008607549086001E000BF00BF00BFDBE098
:1061A00095B90CB10C2100E007210846FCF77EFFF1
:1061B0000CB1032000E00020694908700020694903
:1061C00008606949086000E000BF00BFC4E0052D19
:1061D0007DD2DFE805F0034A6B99AF0063490E7288
:1061E0000846C179072302220420FEF7DFF95F4940
:1061F00091F9060000E0AEE0FFF76CFD5B4991F914
:1062000006105B4A5056FEF75BFE5849C979594A59
:1062100052F82100FEF74EFE5449097A01EB810144
:10622000554A02EB8100FEF751FE504909794F4A69
:10623000527911FB02F101EB8101490001EB4102AE
:10624000C2EBC111494A127A4C4B53F8222002EB9F
:10625000C100FEF729FE45490879FFF729FDC8224C
:1062600000210920FFF786FE73E040490E7109798D
:106270003E4A527911FB02F101EB8101490001EB29
:106280004102C2EBC111394A127A3C4B53F8222029
:1062900002EBC100FEF708FE34490879FFF708FD5C
:1062A000C82200210920FFF765FE52E02F494E71F8
:1062B000497901EB810149004FF47A7211FB02F038
:1062C000FEF7ECFD29490979284A527900E03FE0C0
:1062D00011FB02F101EB8101490001EB4102C2EB2C
:1062E000C111224A127A254B53F8222002EBC10039
:1062F000FEF7DAFD1D490879FFF7DAFCC822002114
:106300000920FFF737FE24E070B21849887191F92F
:106310000610174A5056FFF7DDFC144991F9061094
:10632000134A5056FEF7CCFDC82200210920FFF782
:1063300021FE0EE00D49CE71C9790E4A52F82100B6
:10634000FEF7B8FDC82200210920FFF713FE00E088
:1063500000BF00BF00E000BF00BFBDE8F08100004B
:106360003500002020000020240000203C060020F2
:1063700014650008F864000836000020E86400088E
:1063800010B5574890F90000401EC0EBC00101EB6A
:106390004010544901EB80008E30514991F90010B2
:1063A000491EC1EBC10202EB41114E4A02EB8101D1
:1063B0004968405C002875D0494890F90000401EAB
:1063C000C0EBC00101EB4010114601EB800094309E
:1063D000434991F90010491EC1EBC10202EB411182
:1063E000404A02EB81014968405C08B9012200E0A3
:1063F00000223B4890F90000401EC0EBC00101EBB9
:106400004010384901EB80019431354890F9000083
:10641000401EC0EBC00303EB4010324B03EB800087
:1064200040680A542E4890F90000401EC0EBC0019D
:1064300001EB4010194601EB80009430284991F996
:106440000010491EC1EBC10202EB41111A4602EBDA
:1064500081014968405C30B3214B93F900305B1EE9
:10646000C3EBC30404EB4313144604EB830303F1AF
:1064700040011B4B93F900305B1EC3EBC30404EBDC
:106480004313144604EB83035868154B93F900300B
:106490005B1EC3EBC30404EB4313144604EB8303FA
:1064A0009A6890471BE00E4890F90000401EC0EB30
:1064B000C00303EB40100B4B03EB800000F14001E5
:1064C000074890F90000401EC0EBC00303EB4010EA
:1064D000044B03EB800082684FF0FF30904710BD03
:1064E000B50100201C110020400ECF1980CE341DB4
:1064F00000A1BC33C0CA893688130000881300008D
:10650000881300008813000088130000881300001F
:1065100088130000E2ECF1F6060005070AC9EEDB7D
:10652000DACAD0CED6BDF8BFC6BCBCD3D0CFDEB998
:10653000ABCBBEA1FAA1FBA1FCA1FDA1E80008061E
:1065400040310070444850435048447000002020BF
:106550007E8004848890A0FFA090888404000404B6
:1065600004FF040400FF00007F0000FF0000080C8F
:1065700008F0101106F80000FC0000FF00000010F9
:1065800011111111915F1111111111100000000072
:10659000FC00000000FF00000804F80000000806EE
:1065A000403100212121217F41C1410101002020F2
:1065B0007E8001020418608060180402010002025B
:1065C000423300011111FF1111FF111101000002EE
:1065D00004F804020A32C20202FA0202020024246F
:1065E000257FC5440044330000FF00000000106018
:1065F00080FF00802020202020FF4040400008082D
:1066000008FF080910111111FF11111110002022AB
:1066100041FE80010102C234081462810100202081
:106620002021273CE424242424272020200020406B
:106630008000FF909090909291FE00000000007FFB
:10664000445A61007F49494949497F00000000FFE1
:106650002010E000FF0204C0302844820200000144
:10666000020418600100E01804020100000080002C
:10667000040E1464840404241C06008080000008B6
:10668000484949494949494848407F0000000000BD
:1066900000FC08080808FC000201FE0000000101DF
:1066A00001010101010109050703030101000000C7
:1066B0000000000000002040C080800000000101B8
:1066C00003030705090101010101010101000000A7
:1066D0008080C0402000000000000000000000009A
:1066E0000000020C38FF380C02000000000000001F
:1066F0000000000000FF000000000000000000009B
:106700000000000000FF000000000000000000008A
:10671000000040301CFF1C30400000000000004022
:106720002017081010101010100817204000000249
:1067300004E81008080808080810E804020000002F
:106740000000000000000000000000000000000049
:10675000001F00000000000000CC00000000000846
:10676000304008304000000000000000000000023F
:10677000031E02031E000020FC2020FC2000000E4F
:1067800011113F100C0000180404FF8478000F1052
:106790000F0106180000008C30C078847800000FCC
:1067A00010110E0000007884C43498E48408004876
:1067B0007000000000000000000000000000000069
:1067C000000718204000000000E01804020000400C
:1067D00020180700000000020418E0000000020278
:1067E000010F01020200404080F0804040000000A4
:1067F00000000700000000808080F08080800000A2
:1068000000000000000000090E0000000000000071
:106810000000000000000080808080808000000078
:10682000000000000000000C0C0000000000000050
:106830000000031C2000000618E000000000000714
:1068400008101008070000F008040408F000000019
:1068500008081F00000000000404FC040400000EEF
:10686000101010100F00000C142444840C00000CB5
:10687000101010110E000018048484443800000029
:1068800001020C1F00000060A02424FC2424001F2F
:106890001111111010000098040404887000000702
:1068A00008111109000000F088040404F800001821
:1068B0001010111618000000007C80000000000E6F
:1068C000111010110E000038448484443800000F69
:1068D000101010080700008048444488F0000000B1
:1068E0000003030000000000000C0C00000000008A
:1068F0000001000000000000000700000000000090
:10690000010204081000008040201008040000026A
:1069100002020202020000404040404040000010DD
:106920000804020100000004081020408000000E4E
:10693000121010110E000000000CEC000000030CFF
:10694000131417080700E018E414F414E80000001A
:10695000031C07000000043CC44040E41C04101F5A
:106960001111110E000004FC040404887000030CD3
:10697000101010101C00E018040404081000101F70
:1069800010101008070004FC04040408F000101F95
:1069900011111710080004FC0404C4041800101F8F
:1069A00011111710080004FC0400C0000000030CC3
:1069B0001010101C0000E018040444784000101F60
:1069C000100000101F1004FC84808084FC04001060
:1069D000101F10100000000404FC0404000000005C
:1069E00010101F10100003010101FE000000101F15
:1069F00011031418100004FC0480641C0400101F10
:106A000010000000000004FC040404040C00101F2B
:106A10001F001F1F100004FC807C80FC0400101F5E
:106A20000C0300101F1004FC0400E018FC00070811
:106A3000101010080700F00804040408F000101FEC
:106A4000101010100F0004FC8480808000000708E4
:106A5000101010080700F00814140C0AF200101FA0
:106A6000111111110E0004FC0400C0300C04000EC2
:106A7000111010101C00001C0484844438001810ED
:106A8000101F10101800000004FC04000000101F6C
:106A9000100000101F1000F804040404F800101E79
:106AA000110000131C100000E01C70800000101F7B
:106AB000001F001F100000C07C807CC00000101868
:106AC000160101161810040C34C0C0340C04101C3C
:106AD0001300131C1000000004FC04000000081048
:106AE0001010131C1000041C64840404180000001F
:106AF000007F40404000000000FE02020200002033
:106B00001C030000000000000080601C0300004027
:106B100040407F00000000020202FE000000000072
:106B200020404020000000000000000000000000A5
:106B3000000000000000010101010101010100400D
:106B400040200000000000000000000000000000E5
:106B50000101010000000098242448FC0400080FF3
:106B600000010100000000FC88040488700000009F
:106B70000001010100000070880404048800000086
:106B8000010101090F0000F804040408FC040000DE
:106B900001010101000000F824242424E800000180
:106BA000010709090400000404FC040400000000BB
:106BB00001010101010000D6292929C90600080F99
:106BC00000010101000004FC84000004FC04000139
:106BD000191900000000000404FC04040000000077
:106BE0000001191900000003010101FE0000080F57
:106BF00000000101010004FC2460940C0400000862
:106C0000081F00000000000404FC0404000001014F
:106C100001010101010004FC0400FC0400FC01016D
:106C200000010101000004FC84000004FC040000D9
:106C300001010101000000F804040404F80001014E
:106C400000010100000001FF8904048870000000B9
:106C5000000101000100007088040489FF010101A6
:106C60000100010101000404FC8404008000000014
:106C700001010101010000CC24242424980000011A
:106C8000010701010000000000F8040408000101F0
:106C900000000001010000F804040408FC040101E4
:106CA00001000101010000C0300C30C000000101F2
:106CB00000010100010180700C30E01C60800001C7
:106CC00001010001010000048C70748C04000101BA
:106CD0000100000101010081611E186080000001B7
:106CE00001010101010000840C3444840C00000007
:106CF0000000003F404000000000807C02020000D5
:106D00000000FF00000000000000FF000000404005
:106D10003F000000000002027C80000000000040F4
:106D20008040402040000000000000000000F8F813
:106D30000CC40CF8F00003070C080C07030000104B
:106D400018FCFC0000000008080F0F080800080CE1
:106D500084C4643C18000E0F0908080C0C00080CD1
:106D6000444444FCB800040C0808080F0700C0E0C5
:106D7000B098FCFC8000000000080F0F08007C7C2D
:106D8000444444C48400040C0808080F0700F0F8C9
:106D90004C4444C08000070F0808080F07000C0C83
:106DA0000484C47C3C0000000F0F00000000B8FC0D
:106DB000444444FCB800070F0808080F0700387C5B
:106DC000444444FCF800000808080C0703000000D5
:106DD00000000000000000000000000000000000B3
:106DE00000000000000000000000000000000000A3
:106DF000000000000000000F1F3F7F7F7FFF7F7FAC
:106E00007F3F1F070000000000000000000000009E
:106E10000000000000000000000000000000000072
:106E20000000000000000000000000000000000062
:106E30000000000000000000000000000000000052
:106E4000000000000000000000000101010101013C
:106E50000100000000C0E0F0F8F8FCFCFCF8F8F0DD
:106E6000E0800000010101010101010000000000BB
:106E70000000000000000000000000000000000012
:106E80000000000000000000000000000000000002
:106E900000000000000000000000000000000000F2
:106EA00000000000003F7FFFFFFFFFFFFFFFFFFF2D
:106EB0007F1E000000000000000000000000003FF6
:106EC0007FFFFFFFFFFFFFFFFFFF7F1E00000000AF
:106ED00000000000000000000000000000000000B2
:106EE00000000000000000000000000000000000A2
:106EF00000000000000000000307070F0F0F0F0F36
:106F00000703010080C0E0E0F0F0F0E0F0F8FC7E64
:106F10003F1F0F070F0F0F0F0F0F1F3F7EFCF8F0E3
:106F2000E0E0F0F0F0E0E0C0800000000307070FB1
:106F30000F0F0F0F0703010000000000000000000A
:106F40000000000000000000000000000000000041
:106F50000000000000F8FEFFFFFFFFFFFFFFFFFF44
:106F6000FFF9010000000000000000000000F8FE32
:106F7000FFFFFFFFFFFFFFFFFEFCF8000000000027
:106F8000000000000000010103FFFFFFFFFFFFFF03
:106F9000FFFFFFFEFCF80000000000000000000002
:106FA00000000000010F1F3F3F3F7F7F3F3F3F1F1B
:106FB0000F0100000000008080808080C0E0F0F8B9
:106FC000FFFF7F3F3F7F7F7F3F3F1F0F030000009A
:106FD000808080808000000000070F1F3F3F7F7F80
:106FE0007F3F3F7FFFF3E0C0800000808080808093
:106FF00000000000010F1F3F3F3F7F7F3F3F3F1FCB
:107000000F0180E0F8F8FCFCFCFCFCFCFCFEFF8FB0
:107010000F07030101010101010101010307EFFF56
:10702000FFFEFCFCFCFCFEFFFFFFC70303010001A9
:1070300001010101010307EFFFFFFEFCFCFCFCFC6A
:10704000FCFEFFDF0F07030301010101010103073C
:107050000F1FBFFEFCFCFCFCFCFCFCFCF8F8E08015
:107060000000000000000000000000000080C0FFE1
:10707000FFFFFFFFFFFFFFFFFFFFFFDE80000000BD
:107080000000000000000080C0FFFFFFFFFFFFFFC7
:10709000FFFFFFFFFFDE8000000000000000000097
:1070A000000080FFFFFFFFFFFFFFFFFFFFFFFF9ECE
:1070B00000000000000000000000000000000000D0
:1070C0000000000000000000000000000000C0C040
:1070D000E0F0F0F0F0E0E0C0800000000000000010
:1070E0000000000000000000C0C0E0F0F0F0F0E0A0
:1070F000E0C0800000000000000000000000000070
:107100000000C0C0E0F0F0F0F0E0E0C0800000005F
:10711000000000000000000000000000020603471D
:1071200008050B060D100EA70F6210C7118312136E
:107130001540181819161B4320FB23E9242A2500A3
:10714000261F2C812D352E096871000800000020B3
:1071500010020000BE090008D471000810020020CF
:10716000901700002423000801122B803F047A01AD
:107170000CA183B80BC80F56473232313253343327
:10718000334E30533114FB393014FC383638148CFC
:1071900039313514396E046714080284A24A040098
:1071A00009440102030406070809294C6950051027
:1071B00002040608130D121408F911B9181A6D14F7
:1071C0001A5904193E190201260A26FF2931022FF5
:0471D000C0000000FB
:0400000508000131BD
:00000001FF
